:020000040800F2
:1000000000180020176A0008C56900088D6A0008FA
:10001000C9690008CB690008CD690008000000002C
:10002000000000000000000000000000CF69000890
:10003000D169000800000000D3690008950D000890
:10004000D7690008D9690008DB690008DD69000884
:10005000DF690008E1690008E3690008E569000854
:10006000E7690008E9690008EB690008ED69000824
:10007000EF690008F1690008F3690008F5690008F4
:10008000F7690008F9690008FB690008FD690008C4
:10009000FF690008016A0008036A0008056A000891
:1000A000076A0008096A00080B6A00080D6A000860
:1000B000090E0008116A0008136A0008656100084B
:1000C000034B802252049A61024B04221A6070474B
:0800D00000040048181500208F
:1000D80033230349034A0A60013B002BFBD17047D5
:0800E80000300040AAAA00004C
:1000F000294AD16980239B020B43D3619023DB05FE
:100100001A6850218A431A601A6850310A431A60EB
:100110001A6A22490A401A62196A882252010A435D
:100120001A621F4B1F4A13601F4A13601F4B1B6844
:10013000262B28D00CD9392B2BD0603B5A1E93414B
:100140005B421B4A13409C225201944663440BE0DD
:10015000132B1BD01F3B5A1E93415B42154A134081
:10016000C022D200944663449BB2134A93818023F9
:100170009B025360002393602D3313600F4B80224A
:1001800052051A6070479C23DB00EDE79C231B019E
:10019000EAE7D0239B00E7E700100240FF00FFFFE3
:1001A0000411002000150020FC1400202015002060
:1001B00020EEFFFFA0FBFFFF0044004000E100E055
:1001C00004498022CB691A42FCD080B2014B1885C9
:0801D0007047C04600440040E6
:1001D80010B50400074B1B68002B04D0064B1B68A6
:1001E800002B03D110BDFFF7E7FFF7E7200006F06B
:0C01F80009F8F7E7081500202C1400207F
:1002040010B504004A4B1868C3434A4A1168CA43EC
:100214000140013100D170E0474901200860190C08
:10022400464801601B041B0C45480360002902D1A9
:10023400424944480860002B02D1414B42491960AD
:10024400D107C91706230B400A3340490B604049C4
:100254000B6013065B0E3F490B60002C4CD053051A
:100264009B0F3D490B601304DB0E04333B490B60C9
:10027400120C3B4B1A603B4B1B68DB431A04120CF9
:1002840039490A601B0C394A1360394A1468E4433B
:100294002204120C802109018A4201D935490A43FA
:1002A40035490A60002B2DD1344B354C354819198A
:1002B40004CBD2430A608342F9D1334C3348191931
:1002C40004CBD2430A608342F9D103F059FF264B91
:1002D4001B68002B07D09023DB051B8A1B0702D465
:1002E400214B00221A600D20FFF774FF04F0FAFA84
:1002F4001D4B1B68002B15D110BD04F01DF9002CFB
:10030400E3D1F9E702F098FB02F01CFC240C8023F3
:100314001B019C4201D9174B1C431D4B1C6002F06E
:100324006BFCC1E7013B1B4A136003F037FCE3E7B6
:10033400007400080474000810150020BC14002088
:100344001415002083040000405700007C14002092
:1003540050140020201500205814002060140020A0
:100364005C14002008740008B814002094140020C1
:100374000C7400080000FFFF7814002010740008BB
:100384000094FF17007A00081088FF170080000807
:08039400741400207014002015
:10039C00F0B5C64600B586B001A9294B0A0013CBAF
:1003AC0013C203CB03C2274B01221A60264B002237
:1003BC001A6005F013F9254A254B1A60254B98460F
:1003CC00254F234E254D06E02B68002B13D1204BD7
:1003DC001B68002B0FD043461F6034689442F3D047
:1003EC00A3059B0D1E4922008B42EDD12E20FFF759
:1003FC00EDFE2200E8E701A806F067FB174B1B682F
:10040C00002B0CD06F20FFF7E1FE6B20FFF7DEFE18
:10041C00C82000F079F806B080BCB846F0BD652065
:10042C00FFF7D4FE7220FFF7D1FE7220FFF7CEFE4D
:10043C006F20FFF7CBFE7220FFF7C8FEE8E7C0463F
:10044C0094620008C014002028140020B80B00008F
:10045C000415002000300040AAAA00002C14002033
:04046C00FF0300008A
:1004700010B51E4B1B68002B15D11C4B32221A6085
:100480001B4B1C4A1A601C4B1B68002B0CD0013BF9
:10049000194A1360002B07D0184B1B685A1C132BEA
:1004A00007D0164B1A6010BD154B802252009A617E
:1004B000F2E7124B00221A60124B1B68002BF2D19C
:1004C000114B1A60114B1B681F2B09D0104B1B6876
:1004D000002BE8D1FFF762FF0D20FFF77DFEE2E77A
:1004E0000A4B0B321A60FFF703FEEFE70C150020F2
:1004F00000300040AAAA00001815002010140020A7
:10050000000400482C1400200815002020150020AD
:04051000C0140020F3
:1005140010B5054B1860002805D01C00FFF7A6FF96
:0C0524002368002BFAD110BD1C1500202C
:10053000F8B5D1490122CB681A42FCD1CE4B1B69D8
:100540001B0604D5CC4BCD4A5A60CD4A5A60CA4BE3
:100550001A6902210A431A61CA4A5A611A693E316C
:100560000A431A6119000122CB681A42FCD1C24B1E
:10057000DB689B0604D5C04AD36820210B43D360B7
:10058000BD4B1A6902218A431A611A6901390A436B
:100590001A61BD4B1B68DB43BA4A1380B64901227E
:1005A000CB681A42FCD1B44BDB689B0604D5B24A37
:1005B000D36820210B43D360B44B1B68DB43B44AA0
:1005C0001380AD490122CB681A42FCD1AA4BDB68EB
:1005D0009B0604D5A84AD36820210B43D360AD4BBA
:1005E0001B685B00FF221A40AB4B1B680A3B591E7D
:1005F0008B411A43A94B1B685B02C021C9000B4009
:100600001A43A74B1B68043BDB061B0C1343DB435D
:10061000A44A138098490122CB681A42FCD1964B18
:10062000DB689B0604D5944AD36820210B43D36032
:100630009D4B1B68DB439D4A13808F490122CB6889
:100640001A42FCD18C4BDB689B0604D58A4AD368DE
:1006500020210B43D360964B1B68DB43954A1380E4
:1006600085490122CB681A42FCD1834BDB689B068B
:1006700004D5814AD36820210B43D3608E4B1B687D
:10068000DB438E4A13807C490122CB681A42FCD19D
:10069000794BDB689B0604D5774AD36820210B434E
:1006A000D360874B1B68DB43864A13807249012263
:1006B000CB681A42FCD1704BDB689B0604D56E4AAE
:1006C000D36820210B43D3607F4B1B68DB437F4AF9
:1006D000138069490122CB681A42FCD1664BDB6862
:1006E0009B0604D5644AD36820210B43D360784825
:1006F000784C241A604B01222025774F02E0043009
:10070000B8421AD006190168C9433180D9680A4233
:10071000FCD1D9680D4202D0D9682943D96001685B
:10072000C943090C7180D9680A42FCD1D9680D42CD
:10073000E5D0D9682943D960E1E74F4B1A69012117
:100740008A431A61654A664911601A6902210A439F
:100750001A61644A5A611A693E310A431A611900E2
:100760000122CB681A42FCD1434BDB689B0604D5BF
:10077000414AD36820210B43D3603F4B1A690221C1
:100780008A431A611A6901390A431A6152480122DF
:100790002025554F02E00430B8421AD006190168EE
:1007A000C9433180D9680A42FCD1D9680D4202D0D0
:1007B000D9682943D9600168C943090C7180D96897
:1007C0000A42FCD1D9680D42E5D0D9682943D960E5
:1007D000E1E74648464C241A274B01222025454F85
:1007E00002E00430B84219D006190168C9433180CB
:1007F000D9680A42FCD1D9680D4202D0D968294390
:10080000D9604188C9437180D9680A42FCD1D9684E
:100810000D42E6D0D9682943D960E2E7164B1A6940
:1008200001218A431A612D4A2D4911601A6902215A
:100830000A431A61304A5A611A693E310A431A6101
:1008400019000122CB681A42FCD10B4BDB689B06D6
:1008500004D5094AD36820210B43D360064B1A699B
:1008600002218A431A611A6901390A431A61012275
:100870002025224F47E0C046002002402301674563
:10088000AB89EFCD0074000814150020BC140020C3
:1008900002740008201500207C1400205814002049
:1008A00060140020047400085C1400200674000822
:1008B000B814002008740008941400200A7400087A
:1008C000781400200C740008741400200E740008C2
:1008D0001008002010740008000C002000300040B8
:1008E000AAAA000000780008000E002010020020D4
:1008F000007A000810040020007C00081008002086
:100900000430B84219D006190168C9433180D9684A
:100910000A42FCD1D9680D4202D0D9682943D96076
:100920004188C9437180D9680A42FCD1D9680D4217
:10093000E6D0D9682943D960E2E7064B1A6901215C
:100940008A431A611A697F310A431A610A20FFF744
:08095000E1FDF8BD00200240AA
:1009580070B5041E00DA9CE0092C00D893E0632CE3
:1009680000D881E0FA239B009C426ED3534B9C42F3
:100978005AD9534B9C4248D9524B9C4236D9524B78
:100988009C4224D9514B9C4212D9514B9C4200D9CC
:1009980084E05049200006F04FFB05004D49200037
:1009A80006F0D5FA0C0028003030C0B2FFF710FC72
:1009B8004949200006F040FB05004749200006F0A1
:1009C800C6FA0C0028003030C0B2FFF701FC4349DA
:1009D800200006F031FB05004049200006F0B7FA78
:1009E8000C0028003030C0B2FFF7F2FB3C49200071
:1009F80006F022FB05003A49200006F0A8FA0C0090
:100A080028003030C0B2FFF7E3FB3649200006F07B
:100A180013FB05003349200006F099FA0C00280062
:100A28003030C0B2FFF7D4FBFA218900200006F06D
:100A380003FB0500FA218900200006F088FA0C0063
:100A480028003030C0B2FFF7C3FB6421200006F055
:100A5800F3FA05006421200006F079FA0C0028005A
:100A68003030C0B2FFF7B4FB0A21200006F0E4FAE8
:100A780005000A21200006F06AFA0C002800303030
:100A8800C0B2FFF7A5FB20003030C0B2FFF7A0FBD3
:100A980070BD2D20FFF79CFB64425DE712492000E2
:100AA80006F0CAFA05001049200006F050FA0C00BA
:100AB80028003030C0B2FFF78BFB6AE70F27000031
:100AC8009F8601003F420F007F969800FFE0F505E2
:100AD800FFC99A3B00E1F5058096980040420F0057
:0C0AE800A08601001027000000CA9A3B05
:100AF40070B58CB006AD124B2A0013CB13C213CBC6
:100B040013C26C460F4B220043CB43C243CB43C2B8
:100B14000D20FFF75FFB280005F0DBFF3420FFF713
:100B240059FB2E20FFF756FB2420FFF713FF20006C
:100B340005F0CFFF0D20FFF74DFB0CB070BDC04694
:080B4400A8620008C06200086D
:100B4C0070B54E494A6980239B0213434B614A6935
:100B5C008023DB0213434B619020C005002303600C
:100B6C00474A1360474CC4604748D060D468474D2F
:100B7C002C40D4601068284010601468802040021B
:100B8C00204310608020400090618A69FF38024346
:100B9C008A613F490A680F3002430A603D4A32219C
:100BAC0011603D4A13603D4A13603D4A13603D4A53
:100BBC003D4911603D4A3E4911603E4A13603E4A30
:100BCC0013603E4A13600A223D490A603D490A609F
:100BDC003D4A13603D4B0B221A603D4B3D4A1A6057
:100BEC003D4B1868FA21890006F024FA013880235D
:100BFC005B0498420DD2394A50603948036A1B0293
:100C0C001B0AC02109060B430362002393600733C0
:100C1C0013600A20FFF778FC324C334B2360334BC4
:100C2C00A3600220FFF770FC022363600220FFF731
:100C3C006BFC2F4B23600020FFF7DEFA0220FFF73E
:100C4C0063FCFFF74FFA0220FFF75EFCFFF74CFF47
:100C5C000220FFF759FC274B00221A60FFF798FB84
:100C6C000120FFF7C9FA244C03F0EEFA01F02EF93B
:100C7C002368002BF8D002F0F1FFF5E700100240DA
:100C8C0000040048AAAA0AA4AAAAAAAAFFFFFCFF69
:100C9C00000001400C150020181500201C15002028
:100CAC0004150020BC14002083040000141500203F
:100CBC004057000028140020C014002010150020FC
:100CCC007C14002050140020081500202015002052
:100CDC0068140020A1B0B9120C02002010E000E052
:100CEC0000ED00E00030004055550000FFFF000013
:0C0CFC00CCCC00002C140020441400207C
:100D080010B5FFF7B1FB0F4B1B680F4A12689342EF
:100D180015D05A1C0B490A601B7880200002184322
:100D28000A4B1B689A4207D0094B802252049A61E9
:100D3800084B04221A6010BD074A0A60F4E7002035
:100D4800F9E7C046FC140020001500200802002026
:0C0D5800000400481815002004110020C1
:100D640010B5094B1B68002B05D1084B1B680020EC
:100D7400002B05D010BD05F029F80028F5D0F9E7BF
:100D8400FFF7C0FFF6E7C0462C140020081500202A
:100D9400164B1B68002B02D0013B144A1360144B02
:100DA4001B68002B02D0013B114A1360114B1B68D6
:100DB400002B02D0013B0F4A13600F4B1B68002B22
:100DC40002D0013B0C4A13600C4B1B68002B02D071
:100DD400013B0A4A13600A490A6853035A40530CF8
:100DE40053405A0153400B607047C0460C15002015
:100DF4001C15002004150020881400205414002021
:040E0400681400204E
:100E080010B51A4BDB699B062BD5184B9B8C9BB2F4
:100E1800174A1268002A1AD1FF321A40022A0FD044
:100E2800042A11D0134A11680B7013680133136038
:100E3800114A1268934214D10E4B104A1A6010E0FE
:100E48000F4A02211160EDE700F052FD09E0094A5E
:100E580011680B70136801331360074A12689342D4
:100E680000D010BD034B054A1A60FAE70044004061
:100E78000815002000150020080200200411002099
:040E880048140020EA
:100E8C00024A202311680B4313607047981400200A
:100E9C00064A1368043B1360054A0C32934204D291
:100EAC00044A042311680B43136070476414002038
:080EBC005C13002098140020D3
:100EC400084B1A68111D1960074B5433994202D21A
:100ED400136853607047054A042311680B43136079
:100EE400F8E7C046641400205C1300209814002026
:100EF400044B19680A1F1068096811601B681860A0
:080F04007047C0466414002090
:100F0C00034A1368191D11601A1F12685A60704742
:040F1C006414002039
:100F2000074A1368190008390868043B1B680B60FE
:100F30001368191F1B680B60136818607047C04660
:040F40006414002015
:100F4400074A13681968181F006818601368181F87
:100F5400083B1B6803601368083B19607047C04670
:040F640064140020F1
:100F68000C4B19680A680C4BCB1A9B109B1A042B64
:100F780006D4002A0AD092008A1A13680B607047B8
:100F8800064A042311680B431360F8E70439014B40
:100F98001960F4E7641400205C1300209814002002
:100FA80030B5144B1A681168134BD31A9B105B1A8F
:100FB800042B19D4043A0F4B1A60012913D90123C1
:100FC8005B1A9B009D580222521A9200094C236812
:100FD80098589B18043B1860013904320029F6D14F
:100FE800044B1B681D6030BD044A042311680B4381
:100FF8001360F8E7641400205C13002098140020A4
:10100800F0B5144B1A681568134BD31A9B105B1B69
:10101800042B19D4043A17680E4B1A60012D12D903
:101028006E1E0422524200211C00236898589B1807
:1010380058600131043AB142F7D101235D1B054BD9
:101048001B68AD00EF50F0BD044A042311680B4340
:101058001360F8E7641400205C1300209814002043
:10106800054B1A68111F12680868844662440A60B2
:0C1078001A68043A1A60704764140020E3
:10108400024B1A681368013313607047641400201C
:10109400054B1A68111F12680868821A0A601A68D8
:0C10A400043A1A607047C0466414002033
:1010B000024B1A681368013B1360704764140020E8
:1010C000044B1A681368002B00DB70475B42136007
:0810D000FBE7C0466414002098
:1010D80010B50F4B1B681A68D117501848401F28C5
:1010E80009DC191F0A4C2160002A0BDB0B00096878
:1010F8009140196010BD074A8023DB0011680B433B
:101108001360F7E7043B1A68C2401A60F2E7C0466A
:0811180064140020981400206B
:10112000054B1A68111F1268086802400A601A68A5
:0C113000043A1A607047C04664140020A6
:10113C00054B1A68111F1268086802430A601A6886
:0C114C00043A1A607047C046641400208A
:10115800054B1A68111F1268086842400A601A682D
:0C116800043A1A607047C046641400206E
:10117400024B1A681368DB43136070476414002041
:10118400024B1A6813685B421360704764140020B2
:10119400054B1A68111F1268086842430A601A68EE
:0C11A400043A1A607047C0466414002032
:1011B00010B50B4B1C682168002909D0043C20683D
:1011C00005F020FF2060064A1368043B136010BD41
:1011D000044A80231B0111680B431360F7E7C046E4
:0811E0006414002098140020A3
:1011E80010B50B4B1C68216800290AD0221F106813
:1011F800083C23685843064B1C6005F0FFFE20603E
:1012080010BD044A80231B0111680B431360F7E7E4
:0812180064140020981400206A
:1012200010B50B4B1C682168002909D0043C2068CC
:1012300005F01AFF2160064A1368043B136010BDD5
:10124000044A80231B0111680B431360F7E7C04673
:08125000641400209814002032
:1012580070B50D4B1C682568002D0ED0043C26681F
:101268002900300005F0FCFE2160074B1C682900AE
:10127800300005F0C3FE206070BD044A80231B01C6
:1012880011680B431360F7E76414002098140020DA
:10129800034A1368191D1160024A12685A607047A0
:0812A80064140020681400200A
:1012B000064A1368191F1B6808681B1A58424341E5
:1012C0000B601368043B13607047C0466414002031
:1012D000064A1368191F1B6808681B1A581E8341A9
:1012E0000B601368043B13607047C0466414002011
:1012F000034B1A6811684B424B4113607047C0465C
:041300006414002051
:10130400074B1A68131F012112681868904200DC09
:1013140000211960024A1368043B13607047C046F9
:04132400641400202D
:1013280030B5074B1A68111F10680A68D217C40F26
:101338000D68854262410A601A68043A1A6030BD35
:041348006414002009
:10134C00074B1A68131F012112681868904200DBC2
:10135C0000211960024A1368043B13607047C046B1
:04136C0064140020E5
:10137000064A1368191F1B68086884469C459B41F0
:101380005B420B601368043B1360704764140020D9
:1013900030B5074B1A68111F08681468C20FE517AB
:1013A00084426A410A601A68043A1A6030BDC04635
:0413B00064140020A1
:1013B400044B0A221A60044B1B68002B01D1034B17
:1013C4001A607047501400209C1400207C140020E4
:1013D400044B10221A60044B1B68002B01D1034BF1
:1013E4001A607047501400209C1400207C140020C4
:1013F4000F4B1B68012B05D00E4A402311680B4389
:10140400136070470C4B19680A1D1A600B4B1B685C
:101414000B4A1268934203D005D2D31A4B60F0E70B
:1014240000234B60EDE79B1AC4334B60E9E7C046E9
:10143400081500209814002064140020FC140020D7
:04144400001500206F
:1014480006490A681368043A0A60002B05D0044963
:10145800044A0A60013B002BFBD17047641400204A
:0814680000300040AAAA0000B8
:1014700004490B6864221868424303480260043B35
:0C1480000B60704764140020541400201E
:10148C0010B5054B1C68221D1A60044B18686421AA
:10149C0005F0D0FD606010BD6414002054140020D1
:1014AC0030B5094B1B68013B08495B181B041C0C2D
:1014BC00074802681B0E15684B5513689C4661441F
:1014CC004C70043A026030BDA814002010020020B9
:0414DC006414002074
:1014E000044B1A68111D1960034B1B68043B1B68F1
:0C14F00053607047641400206C1400204E
:1014FC00024B1B681A68024B1A6070476C14002070
:04150C009014002017
:10151000064B1B681A68002A04D1054A1268116834
:10152000044A1160043B014A1360704764140020B0
:081530006C140020901400204F
:10153800154B1B68154A19681160154A934218D94A
:10154800144A1268022A07D0043B0F4A1360124A51
:101558001368013B136070470F4A11680F4A1268FD
:101568009142F1D10D4A002111600A4A03311160FC
:10157800EAE7064B00221A60064B1B68022BEAD1E9
:10158800044B03321A60E6E76C1400209014002024
:10159800F8120020FC01002084140020B41400205C
:1015A800054B00221A605A609A6018000C300349F3
:1015B8000860DA607047C0465C130020641400209D
:0C15C800014B03221A607047FC01002058
:0C15D400014B01221A607047FC0100204E
:0C15E000014B00221A607047FC01002043
:1015EC0030B50D4B1C68221D1A600C490B685A1C37
:1015FC000A60587800069A1C0A609A781204024312
:10160C00D81C0860D87800021D1D0D601B7913438F
:10161C000343636030BDC046641400209014002066
:10162C00054A1368191D116004490A68501C0860AA
:10163C0052785A607047C046641400209014002001
:10164C00074B19680A1D1A60064A1368581C10606B
:10165C005A781201044B9B189B684B607047C0462C
:0C166C00641400209014002010080020DE
:10167800074B1A68511C196006480368517809011C
:10168800054A521819689160043B03607047C046C8
:0C169800901400206414002010080020B2
:1016A400074B1A68511C196051780902901C186084
:1016B40092781143802292050A431A607047C0460B
:0416C400901400205E
:1016C80010B5094B1868021D1A6008490B685A1CA6
:1016D8000A605A7812029C1C0C609B781A4380237B
:1016E8009B051343436010BD6C1400209014002028
:1016F800084B094A1A60094B1A68511C196051783D
:101708000902901C186092781143802292050A43BE
:101718001A60704700300040AAAA00009014002008
:1017280010B5094B1B681A68023A80239B051343BE
:101738001A78752A03D1013B044A136010BD034A85
:101748001360FFF7D5FFF9E76C1400209014002010
:1017580010B50A4B1B681B68002B0CD0084A13688D
:10176800043B1360074A136803331360034A136882
:10177800043B136010BDFFF7BBFFF7E764140020BC
:081788006C14002090140020F5
:1017900010B50A4B1B681B68002B0CD1084A136854
:1017A000043B1360074A136803331360034A13684A
:1017B000043B136010BDFFF79FFFF7E764140020A0
:0817C0006C14002090140020BD
:1017C80010B5104B1A681100103119600E490B68DA
:1017D800180008380068D060181F00689060186802
:1017E80050600C3B0B6009480368591C016059782C
:1017F80009029C1C04609B78194380239B050B43BA
:10180800136110BD6C140020641400209014002093
:1018180010B5254B1B681A1F12681900083908688B
:101828000C3B19685318214A214C146000291DDB10
:10183800984212DD1C4A1268043A13601D4B1A685C
:10184800511C196051780902901C18609278114354
:10185800802292050A431A6010BD134A1368103B90
:101868001360144A136803331360F5E7984212DAD9
:101878000D4A1268043A13600E4B1A68511C19601D
:1018880051780902901C18609278114380229205C1
:101898000A431A60E0E7044A1368103B1360054ADC
:1018A800136803331360D7E76C140020003000403E
:0818B800AAAA00009014002010
:1018C000024A1368043B13607047C0466C14002042
:1018D000024A1368103B13607047C0466C14002026
:1018E00010B5044C23681878FEF776FC2368043B97
:0818F000236010BD6414002008
:1018F80000B583B06A46094B03CB03C2084B1B688B
:10190800002B01D003B000BD684605F0E0F8044B99
:1019180001221A60034B00221A60F3E7D86200081C
:08192800FC010020481400201E
:1019300010B5114B1B68002B12D0104B1B78002BDD
:101940000ED00F4B1B68002B15D00E4A1368191DC3
:1019500011600D4A12785A60094B00221A600AE0A1
:10196000FFF700FA0028FBD0064B1A68111D19601A
:10197000FF231840506010BDFC0100202B150020F3
:0C1980004C140020641400202A150020E4
:10198C0010B50E4B1B68102B08D00D4B1B6818683C
:10199C00E0231B06C2180B4B9A420CD8084B1B6851
:1019AC00186805F01DFB2020FEF710FC044A136894
:1019BC00043B136010BDFEF7C9FFF4E75014002080
:0819CC0064140020FF0B06303B
:1019D40010B5064C2368186805F006FB2020FEF7B6
:1019E400F9FB2368043B236010BDC0466414002047
:1019F400F0B587B003AA2A4B13CB13C2294B1A683C
:101A040001929A8801AB9A805B20FEF7E3FB264B98
:101A14001B68264A0C3293420DD0244A0C3293425E
:101A24000DD3224A0C32934216D9204C103404258B
:101A34001E4F160024E001A805F04BF80CE003A8A3
:101A440005F047F8194B00221A605A609A60180092
:101A54000C3015490860DA605D20FEF7BBFB2020DE
:101A6400FEF7B8FB07B0F0BD206805F0BDFA2020F2
:101A7400FEF7B0FB01350C4B1B680434B342EBD9C1
:101A8400DB1B9B10AB42E7D32020FEF7A3FB084BE4
:101A94001B68102BE8D02068FEF75CFFE7E7C04620
:101AA400A86A0008B46A0008641400205C130020CB
:041AB40050140020AA
:101AB800F0B5D6464F464646C0B584B001AA394B64
:101AC80003CB03C21B7813702020FEF781FB364B33
:101AD8001B68002B5BD0354D00270026C0231B0553
:101AE8009946334B9A46304B984616E02020FEF72D
:101AF8006FFB14E06B684A46134221D12020FEF7A1
:101B080067FB2020FEF764FB01360137052F34D828
:101B1800103543461B68B34237D9092EE6D9300041
:101B2800FEF716FF3A20FEF753FB2C00083C2078FE
:101B38000028DFD0FEF74CFB0134AC42F7D1D9E7DF
:101B480001A804F0C4FF53461B68102B11D0286865
:101B5800FEF7FEFE2020FEF73BFB4020FEF738FB99
:101B68002804000C05F03EFA2920FEF731FB023765
:101B7800C4E7286805F036FAECE70D20FEF728FBE5
:101B88002020FEF725FB0027C2E7002F05D104B06F
:101B9800E0BCBA46B146A846F0BD0D20FEF718FBDA
:101BA800F5E7C046F06C00088014002018080020F3
:041BB80050140020A5
:101BBC0010B5044C2368186805F035F82368043B0D
:081BCC00236010BD6414002029
:101BD40010B5074B1B68002B04D1064A1368043B5D
:101BE400136010BD034B1B681878FEF7E7FAF4E79F
:081BF400081500206414002014
:101BFC00F0B5C64600B5114A13681F68043B136064
:101C0C00002F13D00125ED1BAD003C000C4E90466F
:101C1C0003E0013C0435002C08D03368002BF8D0CD
:101C2C0043461B68585DFEF7C5FAF2E7034BBF004D
:101C3C001A68D71B1F6080BCB846F0BD6414002026
:041C4C000815002057
:101C5000F0B5C64600B582B06846214B020012CBF3
:101C600012C204F038FF0D20FEF7B6FA1D4DFC231A
:101C70009B009846A8440026012723E0FEF7ACFA13
:101C80000134285D0028F9D1062C05D82020FEF764
:101C9000A3FA0134072CF9D12320FEF79DFA38006E
:101CA00004F041FF2020FEF797FA2020FEF794FA77
:101CB0002020FEF791FA01370136052E07D00835AE
:101CC000A84509D02020FEF787FA0024D9E70D2087
:101CD000FEF782FA0026F2E702B080BCB846F0BDFB
:081CE000E0620008BC65000889
:101CE80070B5FFF73BF8041E00D1D8E0C0B2704BC6
:101CF8001B68002B08D06F4B1B78002B04D06E4B51
:101D080018706E4B01221A600A2800D1C4E002281C
:101D180000D8C3E0674B1B78002B08D109281FD0D7
:101D2800674A12683F2A02D9202800D19EE0282855
:101D380018D02F2840D01B2868D10024002B00D1B0
:101D4800ADE00E38FEF744FA5D4B1A685D4B202172
:101D580099549B18002159705B4B1A6002349EE01D
:101D68001730DDE7594B1C68002C01D0002496E0A1
:101D7800FEF72EFAFEF7F2FF0028FBD0C0B22028AB
:101D88000BD04F490B684F4A2825D554D2185070AC
:101D980002330B60FEF71CFA81E0494B1B680133E4
:101DA8004A4A13601838FEF713FA2020FEF710FA93
:101DB8000820FEF70DFA72E0444B1C68002C01D095
:101DC80000246CE0FEF704FAFEF7C8FF0028FBD0F9
:101DD800C0B22F280BD03A490B683A4A2F25D55460
:101DE800D218507002330B60FEF7F2F957E0344B0B
:101DF8001B680133354A13602738FEF7E9F92020BC
:101E0800FEF7E6F90820FEF7E3F948E0092848D08C
:101E1800122848D0082817D12C4B1D680024002D03
:101E28003DD1274B1C68002C39D0013C1C60254B48
:101E380020221A55FEF7CCF92020FEF7C9F9082010
:101E4800FEF7C6F92C002AE00D2817D11C4B1B6899
:101E5800002B0BD11A4B1A681A4B202199549B1846
:101E680000215970184B1A60012418E0174B1B68A1
:101E7800012BEFD00D20FEF7ABF9EBE7134B1C68F5
:101E8800002C12D10E4D0F4B2A689854FEF7A0F97A
:101E98002B6801332B6002E0002400E000242000BE
:101EA80070BD0324FBE70424F9E70024F7E7C046E4
:101EB800FC0100202B1500202A1500204C140020BE
:101EC800401400209412002044140020A014002084
:101ED80010B50023054A1360054A1360054A1360CC
:101EE800FFF7FEFE0028FBD010BDC04640140020BE
:081EF80044140020A014002096
:101F000010B5154B1968154B5A5C202A09D14B1C8A
:101F10001248013819000133C25C202AFAD00E4B56
:101F200019600023002A10D00C4840180C4CC25CE9
:101F3000202A03D01A5501330F2BF8D1084A00206C
:101F4000D0545B18074A136010BD054B00221A706D
:101F5000044B1960F8E7C0463814002094120020A2
:081F6000C01300204014002012
:101F6800F0B5DE46474680B587B00E0002AA0024C9
:101F780005E0002B1BD001340132102C08D0035D82
:101F88001370190061391929F3D8203B1370F2E74F
:101F9800002302AAD37313782D2B0ED1254B0022D0
:101FA8001A6001239B460127012C0FD82CE000233F
:101FB80002AAD37313782D2B2CD01E4B00221A6043
:101FC80000239B4600270120002C2DD0194B1D68AB
:101FD800B84602AB9C46E044002301934346187878
:101FE800310004F02EFE431C18D075432D1801371C
:101FF80001239C46E0440193A742EFD30D4B1D609B
:1020080001205B46002B0FD00A4A13685B4213601D
:10201800012009E00020012CC0D105E0019B002B24
:1020280001D0044B1D60002007B0C0BCBB46B046C1
:08203800F0BDC0463C1400207D
:1020400010B5344B187800285AD000233149013399
:102050005A5C002AFBD12D280FD0302829D12D4AD7
:10206000527820218A43582A11D02B4A116810290E
:102070003AD1082B48D900204BE0012B3AD0264A10
:10208000116810292AD00B2B3ED9002041E0214AAB
:1020900092782D2A09D00A2B2ED81E481021023002
:1020A000FFF762FF431E984133E00B2BF5D9002068
:1020B0002FE02528D9D1174A52782D2A09D00B2B89
:1020C0001CD814480A210130FFF74EFF431E9841E7
:1020D0001FE00C2BF5D900201BE000232D28C8D1D0
:1020E000092B11D9002014E02D28CCD000200A2B78
:1020F0000FD809E000200CE000200AE0002008E0F2
:10210000054B19681029E8D00248FFF72DFF431E40
:0C211000984110BDC013002050140020A6
:10211C00F0B51A4C00251A4E0021635C8A5D18003C
:10212C00613819280DD8203BDBB210006138192812
:10213C0011D8203AD2B2934219D101310829ECD1ED
:10214C0015E01000613819280DD918002038471EE9
:10215C00B84140420340934209D1002AEDD1094BCA
:10216C001D600120F0BD203AD2B2202BE3D1013505
:10217C0008347F2DD0D10020F4E7C046B4650008A8
:08218C00C013002070140020B4
:1021940070B51A4B1B78002B29D0194A00231E0056
:1021A400013310321100103909780029F7D1731C5A
:1021B4001FD03301114C1C19124D16E08B4211D162
:1021C40000290BD00132082A0CD0A15C535D180001
:1021D40061381928F2D8203BDBB2EFE70A4B1E60C6
:1021E400012070BD103C013E05D30022EDE7002024
:1021F400F7E70020F5E70020F3E7C04610080020C9
:0C22040020080020C013002070140020EF
:1022100010B50F4B1A680F4B1A60FFF771FEFFF7EE
:10222000B9FF002805D00C4B1B6801330B4A136023
:1022300010BD0B4B1B78302B05D00A4A21231168A7
:102240000B431360F4E7054B00221A60F0E7C04629
:10225000401400203814002070140020B81400200E
:08226000C013002098140020B7
:10226800074A13680749C85401331360064A934262
:1022780004D9064A202311680B4313607047C046EF
:10228800A814002010020020FE0500009814002069
:1022980010B5144B18688200134BD3581A030AD48C
:1022A800124A1268002A13D19B030BD48000104BEA
:1022B800C358984705E00F4A80239B0011680B43D9
:1022C800136010BD0B4A082311680B431360F8E72D
:1022D800DB0304D58000064BC3589847F1E7FFF7A6
:1022E800BFFFEEE770140020B86300089C140020BC
:0822F8000000002098140020F2
:1023000070B594B00CA9414B0A0013CB13C213CB88
:1023100013C203CB03C205A93D4B0A0013CB13C262
:1023200013CB13C21B7813706A463A4B13CB13C2FC
:1023300011001A680A601B790B71374B1B68522B0E
:1023400009D95224354E344DA05DFDF745FF0134C7
:102350002B68A342F8D85223314A1360314A002136
:102360001160314A13602E4D304E03E02C4B1A6839
:102370002D4B1A60284C2B682268934234D2FFF709
:10238000BFFD3378002BF6D0FFF75AFE00280BD0A4
:10239000274B1A68274B1A60274B1B78002BE5D078
:1023A000264B01221A60E1E7FFF7B8FE002811D0A2
:1023B000234B1B689B00234A9B585B0321D5FFF7E7
:1023C0006BFF214B1B68002B08D1154B1A68164B6D
:1023D0001A60CFE70CA804F07EFB05E01A4B002240
:1023E0001A60684604F077FB0D20FDF7F5FE5223D6
:1023F000094A13600A4A13600A4B00221A6014B09B
:1024000070BD05A804F067FBEEE7C046086D000844
:10241000286D0008446D0008441400209412002028
:1024200040140020A014002038140020C013002005
:102430003C140020AC1400202B150020B014002008
:0C24400070140020B863000898140020FD
:10244C0070B56F20FFF70AFF0C4D2C68FF20FFF7CB
:10245C0005FFFF20FFF702FF2B68013B084A9B1882
:10246C001B04180C074909681B0E0D6853550B68A3
:10247C009C46624450700C6070BDC046A81400208D
:08248C0010020020641400207E
:1024940010B57020FFF7E6FE064A1368191D116097
:1024A400054A12685A60FF20FFF7DCFEFF20FFF7A1
:0C24B400D9FE10BD64140020A814002004
:1024C00010B57420FFF7D0FE064A1368191D11607D
:1024D000054A12685A60FF20FFF7C6FEFF20FFF78B
:0C24E000C3FE10BD64140020A8140020EE
:1024EC00F8B57520FFF7BAFE104E33681D6801353C
:1024FC000F4C2D19280AFF273840FFF7AFFE380084
:10250C002840FFF7ABFE0B4B1B68013B1B193268D5
:10251C00190A106821541268A41863707720FFF709
:10252C009DFE3368043B3360F8BDC0466414002044
:08253C0010020020A814002089
:1025440010B51F4B1B68002B17D11E4B1B681E4A6E
:10255400196811601D4A93422ED91D4A1268022A35
:102564001DD0043B174A13601A4A1368013B1360D9
:10257400194B1A68194B1A6010BD6420FFF772FEDC
:1025840000220F4B1A6016490B6801330B601B01C4
:1025940014495A54144B1A68144B1A60E8E70D4A4C
:1025A4001168134A12689142DBD1114A002111606B
:1025B400074A03311160D4E7034B00221A60D7E7BE
:1025C4009C1400206C14002090140020F8120020A9
:1025D400FC010020841400207C14002050140020EE
:1025E4008014002010080020A8140020A414002047
:0425F400B4140020FB
:1025F80070B5324B1B68002B27D1314B1B681C78F8
:1026080023005F3B022B16D97D20FDF7E1FD20203A
:10261800FDF7DEFDFFF7EAF92500703D072D15D916
:10262800743C012C1CD9032D0FD8264B1B68188825
:1026380004F0A2FC09E0244B186801300005000DE5
:1026480004F09AFC2920FDF7C3FD70BD2020FDF79A
:10265800BFFD5220FDF7BCFD3A20FDF7B9FDDFE7CD
:10266800184B1A68194BD31A082BEED90C3A108854
:1026780004F082FC2020FDF7ABFD2020FDF7A8FD2B
:10268800104C2368083B188804F076FC2020FDF7DE
:102698009FFD6920FDF79CFD2368043B188804F022
:1026A8006BFC2020FDF794FD7820FDF791FD236851
:1026B8001888013004F060FCC7E7C0469814002071
:1026C8008C1400206C14002090140020F8120020B4
:1026D800104B1B68002B0BD00F4B18680F4B1B6857
:1026E800984205D001D2181A13E0C01AC43010E07D
:1026F8000B4B186800280BD10A4B1B680A4A126852
:10270800934206D0D01A934203D3981AC43000E0FB
:10271800002070472C140020CC140020D014002076
:0C27280008150020FC1400200015002003
:1027340010B5094B1C68221D1A60084B1B68002B3E
:1027440006D0074B1B78002B02D0064B186801E01B
:10275400FFF7C0FF606010BD64140020FC0100207E
:082764002B1500204C1400208D
:10276C0010B50B4B1C6800230A4909190A48CA5CAE
:10277C00222A03D01A5401334E2BF8D1064A2221B7
:10278C00D15401330021D154E318044A136010BD15
:10279C003814002094120020C01300204014002094
:1027AC001A4B1B185A781300613B192B03D8203A8B
:1027BC001300373B05E02F2A1BD91300303B092BA4
:1027CC00F6D80F2B18D8114A1018827811006139DD
:1027DC00192907D8203A373A11000F2912D81801B5
:1027EC00401870472F2A0AD9110030390929F4D919
:1027FC00F1E701204042F4E701204042F1E70120DB
:10280C004042EEE701204042EBE7C046C0130020F7
:10281C00F0B5C64600B50700404B1B680133404A73
:10282C001360FFF79DFF002600243E4A03E00136AB
:10283C000134502C10D0A35C5C2BF8D0222BF7D198
:10284C00384B00221A55384B1D68002D0CD1354CD5
:10285C00364B98461E003BE0354A022311680B4369
:10286C00136080BCB846F0BD012F0ED06620FFF778
:10287C00F5FC304A13687600A41B2F49CC54013365
:10288C0013600024274D2E0009E06520FFF7E6FCBD
:10289C00EFE7FFF7E3FC0134335D002BE1D0285D5B
:1028AC005C28F6D12000FFF77BFF431C03D00334D8
:1028BC00FFF7D4FCF0E71E4A022311680B431360A8
:1028CC00CFE7FDF783FC0135164B5B5D002BC8D0C1
:1028DC00605D5C2807D0012FF3D03368002BF2D059
:1028EC00FDF768FCEFE72800FFF75AFF431C0AD0FE
:1028FC000335012F0DD043461B68002BE4D0C0B22A
:10290C00FDF758FCE0E70A4A022311680B431360F9
:10291C00A7E7C0B2FDF75AFCD6E7C046401400202A
:10292C0038140020C01300209C140020081500202F
:0C293C0098140020A814002010020020B5
:1029480010B5154B1B68022B17D0144B18680028BC
:1029580017D0134B1B780020002B12D0FFF7B8FEBE
:1029680000280ED0FFF7BCF901280BD002280CD0A4
:102978000C4B1868431E984103E0074B00221A606D
:10298800012010BDFFF7B8FCF2E7064A80235B0080
:1029980011680B431360EBE748140020FC0100208A
:0829A8002B15002098140020FB
:1029B00010B50D4B1B68012B05D00C4A4023116844
:1029C0000B43136010BDFEF79FF9002804D1FFF7F9
:1029D000BBFF0028F7D0F5E7054B1A68111D1960F9
:1029E000FF2318405060EDE70815002098140020E0
:0429F000641400204B
:1029F40010B5094A1368094918680860043B136054
:102A04000C002368002B05D0FDF730FDFFF79AFF7B
:102A14000028F6D010BDC04664140020881400209D
:102A240010B5044B1A68642311684B431360FFF715
:082A3400DFFF10BD6414002057
:102A3C0070B5394B1B6880225202934231D3364B0E
:102A4C00364A1A60364B1B88DB0711D4344B0022F4
:102A5C001A821A803349CA6902200243CA61324A77
:102A6C001A83FA22D200DA621A8801210A431A80E8
:102A7C00294B1B68013B9BB2294A13852B4B1B68C6
:102A8C00002B3DDB264A138C01210B431384284B6E
:102A9C001B68002B39DB224A138C10210B43138447
:102AAC002DE0002BCED11E4A13880125AB43138099
:102ABC00012464421D4B1C609023DB0518681D4EDD
:102ACC0030401860D9683140D960D86880218901BC
:102ADC000143D960118CA943118415490C60186805
:102AEC00154C20401860D9682140D960D8688021E5
:102AFC0009020143D960138C10218B43138470BDE0
:102B0C00138C01218B431384C1E7054A138C1021CC
:102B1C008B431384F3E7C04694140020FFFF00009E
:102B2C000004004000100240606000007814002097
:0C2B3C0074140020FFCFFFFFFF3FFFFFDD
:102B48009022D205136827490B401360264A138C3C
:102B580001218B431384254B1B68002B24DB902118
:102B6800C905CA681F480240CA60002B24D0FA224F
:102B7800D20093422ADA9023DB0519688022920159
:102B88000A431A601A6A1A490A401A62196A8022A4
:102B980052040A431A62144B1A8C01210A431A84FC
:102BA800124A12685A6370479022D205D16880236E
:102BB8009B010B43D360F6E70B00096880225201A2
:102BC8000A431A608022D2039A61ECE7074B1A6025
:102BD8009023DB051968802252010A431A604022BB
:102BE8009A61E0E7FFCFFFFF00040040781400205F
:042BF800FFFFFFF0EC
:102BFC009022D205136827490B401360264A138C88
:102C0C0010218B431384254B1B68002B24DB902154
:102C1C00C905CA681F480240CA60002B24D0FA229A
:102C2C00D20093422ADA9023DB0519688022120223
:102C3C000A431A601A6A120112091A62196A80226E
:102C4C0052050A431A62144B1A8C10210A431A8437
:102C5C00124A12689A6370479022D205D168802379
:102C6C001B020B43D360F6E70B0009688022D201EC
:102C7C000A431A60802212049A61ECE7074B1A602F
:102C8C009023DB0519688022D2010A431A60802246
:102C9C009A61E0E7FF3FFFFF00040040741400203E
:102CAC00134A13681868043B136011281DD0F023D5
:102CBC000340A02B0AD00E280AD9B12814D00D4AF3
:102CCC008023DB0011680B4313600DE0913B18402F
:102CDC00831E012B02D9063B042B05D8054A802301
:102CEC00DB0011680B4313607047B120FCE7C04652
:082CFC0064140020981400206C
:102D040010B5FFF7D1FF104B1B68002B0FD10F2814
:102D14000ED89023DB051B8A0122824013400B4905
:102D24000A68101D0860002B0AD00123536010BDEF
:102D3400074B1B8A0F2210400E3A82401340EEE7E5
:102D440000235360F3E7C046981400206414002065
:042D5400000400482F
:102D580006280FD007281AD10D4B1B68013316D04F
:102D68000C4A138C10218B431384094B01225242C5
:102D78001A600CE0084B1B68013308D0054A138C15
:102D880001218B431384044B012252421A6070477D
:0C2D980074140020000400407814002097
:102DA40070B5FFF781FF0400154B1B68002B0FD192
:102DB4000F280ED9134BDA680C218A43DA601A689B
:102DC4008A431A601A6808390A431A6002229A610F
:102DD40070BDFFF7BFFF6000032282409023DB0534
:102DE400D9689143D9601968914319601D6801221B
:102DF4001100814029431960A2409A61E8E7C04666
:082E04009814002000040048AE
:102E0C0070B5FFF74DFF0400164B1B68002B10D15B
:102E1C000F280FD9144BDA680C218A43DA601A6830
:102E2C008A431A601A6808390A431A60802292028F
:102E3C009A6170BDFFF78AFF6000032282409023E5
:102E4C00DB05D9689143D9601968914319601D68F5
:102E5C00012211008140294319601034A2409A616B
:0C2E6C00E7E7C04698140020000400486E
:102E780010B5FFF717FF0400124B1B68002B0DD18C
:102E88000F280CD9104B1A680C218A431A60DA688B
:102E98008A43DA60DA6808390A43DA6010BDFFF756
:102EA80057FF64000322A2409023DB051968914371
:102EB8001960D9689143D960D9680122A2400A43B0
:0C2EC800DA60EBE79814002000040048DA
:102ED40010B5FFF7E9FE0400124B1B68002B0DD15F
:102EE4000F280CD9104B1A680C218A431A60DA682F
:102EF4008A43DA60DA6804390A43DA6010BDFFF7FE
:102F040029FF64000322A2409023DB051968914342
:102F14001960D9689143D960D9680222A2400A4352
:0C2F2400DA60EBE798140020000400487D
:102F300010B5FFF7BBFE04000E4B1B68002B09D138
:102F40000F2808D90C4B1A680C218A431A60DA68DA
:102F50008A43DA6010BDFFF7FFFE64000322A2403F
:102F60009023DB05196891431960D9689143D960B2
:0C2F7000F0E7C046981400200004004860
:102F7C0010B5144BDA6814490A40DA60996980225A
:102F8C0092000A439A61FDF7A1F8FDF79FF8FDF74F
:102F9C009DF8FDF79BF80D4B802212061A6100225A
:102FAC00DA600B490A6004325A619A6801210A43BB
:102FBC009A60190001220B681A42FCD0FDF786F8C2
:102FCC0010BDC04600100240FFFDFFFF0024014071
:042FDC000827014081
:102FE0000C4B1A6801210A431A609A6801310A439E
:102FF0009A60190001228B681A42FCD1064B9A692B
:1030000006490A409A61D968802292000A43DA6030
:103010007047C0460024014000100240FFFDFFFF42
:10302000F0B589B004AA5C4B13CB13C21B88138084
:103030006A465A4B13CB13C21B781370584B1B684C
:103040001C68621C18D0072C03D92300A03B072B57
:103050001BD8544B9B699B051ED5534B534A1A6092
:103060000F232340590003228A40072B00D98BE00D
:1030700099004F4841588F46043B494A1360FFF777
:10308000AFFF684603F027FD35E04A4A8023DB00A6
:1030900011680B4313602EE0FFF770FF04A803F0E4
:1030A0001AFDDAE79021C905086810430860C8686E
:1030B0009043C86001229A4013003B4A9362042661
:1030C000002714000425A3682B43A36023681D4236
:1030D000FCD0236CFF18FCF7FFFF013E002EF2D15D
:1030E0002F4B1B68BA081A60BB0704D52C4B1A6813
:1030F00013680133136009B0F0BD9021C905086859
:1031000010430860C8689043C860D3E79021C905A0
:10311000086810430860C8689043C860CAE79021F7
:10312000C905086810430860C8689043C860C1E7D3
:1031300021490968013108D02048018C0124A143AC
:1031400001841D490120404208609021C90508689A
:1031500010430860C8689043C860ABE71849096825
:10316000013108D01548018C1024A1430184144971
:103170000120404208609021C9050868104308609A
:10318000C8689043C86095E70A4A8023DB0011684D
:103190000B431360AFE7C046646D0008746D000810
:1031A000641400200010024000240140FF070000CA
:1031B000E862000898140020781400200004004001
:0431C0007414002063
:1031C4001B4B1B68032B26D81A4B1B68043B1C2B78
:1031D40021D880235B02184A12689A421BD290239A
:1031E400DB051A6815490A401A60196882225200E0
:1031F4000A431A60DA6803218A43DA60DA6801391B
:103204000A43DA600A4B1B68012B0BD99023DB05B8
:1032140002229A6105E00A4A8023DB0011680B430D
:10322400136070479023DB05802292029A61F8E7CD
:1032340058140020601400205C140020F0FCFFFFF0
:0432440098140020BA
:1032480010B50A4A13680A4918680860191F1160FE
:1032580008680849086019000839116008680649B3
:1032680008600C3B1360FFF7A9FF10BD6414002031
:0C3278005C14002060140020581400209A
:10328400F8B5DE4657464E464546E0B59023DB0585
:103294001B68B94A13408222520093421ED1B74B95
:1032A4001B681C68B64B1A68B64B1868002800D017
:1032B4006FE09023DB05802189029961B24B1B6882
:1032C400002B0ED101259021C905802040038046A2
:1032D400102084468027BF02022643E0FFF770FFD8
:1032E400DDE701239B469025ED0580235B039A4689
:1032F4001023994680239B029846A34B9C46A349DE
:103304001F001DE05346AB614346AB6163461B6837
:10331400002B04D09E4E3160013B002BFBD14000BA
:103324002B8A5E46334018430223AB613B68002B73
:1033340004D0974E3160013B002BFBD1002A1AD0F8
:10334400013A5B4693401C42DCD04B46AB61DBE761
:10335400404688618F615B00088A284003438E6180
:10336400002A07D0013A280090400442F0D0604679
:103374008861EFE718009023DB05802292029A61AE
:103384007E4B1B681860F0BCBB46B246A946A046FB
:10339400F8BD012816D0022879D09023DB0502213C
:1033A4009961794B1868002800D0D3E00125902357
:1033B400DB0580214903884610218C468027BF0203
:1033C400022617E19023DB058021890299616E4B67
:1033D400186800280BD101259023DB0580214903BF
:1033E400884610218C4602278026B60241E0002040
:1033F40001239B469025ED0580235B039A46102309
:1034040099460E3B9846604B9C4660491F001EE05F
:103414005346AB614346AB6163461B68002B04D043
:103424005B4E3160013B002BFBD140002B8A5E4692
:103434003340184380239B02AB613B68002B04D0CC
:10344400534E3160013B002BFBD1002A19D0013AC5
:103454005B4693401C42DBD04B46AB61DAE7414606
:1034640099619F614000198A294008439E61002A9E
:1034740007D0013A290091400C42F0D0614699618D
:10348400EFE79023DB05802292029A6178E790238C
:10349400DB05022199613C4B186800280BD10125FA
:1034A4009023DB0580214903884610218C4602279E
:1034B4008026B60241E0002001239B469025ED05BD
:1034C40080235B039A46102399460E3B98462E4B65
:1034D4009C462E491F001EE05346AB614346AB6138
:1034E40063461B68002B04D0294E3160013B002B3E
:1034F400FBD140002B8A5E463340184380239B0255
:10350400AB613B68002B04D0214E3160013B002BA2
:10351400FBD1002A19D0013A5B4693401C42DBD010
:103524004B46AB61DAE7414699619F614000198AD5
:10353400294008439E61002A07D0013A290091409E
:103544000C42F0D061469961EFE79023DB0502223B
:103554009A6115E7002001239B469025ED05802301
:103564005B039A461023994680239B029846064B98
:103574009C4606491F002BE00F0300006414002042
:1035840060140020581400205C140020AAAA000033
:10359400003000405346AB614346AB6163461B6851
:1035A400002B04D01A4E3160013B002BFBD14000AC
:1035B4002B8A5E46334018430223AB613B68002BE1
:1035C40004D0134E3160013B002BFBD1002A19D0EB
:1035D400013A5B4693401C42DCD04B46AB61DBE7CF
:1035E400414699619F614000198A294008439E61C0
:1035F400002A07D0013A290091400C42F0D06146DC
:103604009961EFE79023DB0502229A61B8E6C04690
:043614000030004042
:1036180010B5074A1368191D1160064A12685A60E6
:10362800FF20FEF71DFEFF20FEF71AFE10BDC04664
:0836380064140020A814002016
:10364000F8B5104E33681D6801350F4C2D19280A46
:10365000FF273840FEF708FE38002840FEF704FE3A
:103660000A4B1B68013B1B193268190A1068215468
:103670001268A41863707620FEF7F6FD3368043BE9
:103680003360F8BD6414002010020020A81400204C
:1036900070B57E280DD8C0000E4D441908352D1880
:1036A0002078002804D0FCF797FD0134AC42F7D114
:1036B00070BD7F2528400001074D441908352D189D
:1036C00020780028F4D0FCF787FD0134AC42F7D114
:0C36D000EEE7C046B465000810080020BA
:1036DC0070B50001064D441908352D1820780028C6
:1036EC0004D0FCF773FD0134AC42F7D170BDC04679
:0436FC001008002092
:10370000F0B5C64600B582B0A34B1A6800929B88FC
:103710006A469380A14B1D68002D03D002B080BC87
:10372000B846F0BD9E4B1B689E4A13601B789846B6
:103730001F009D4B1B685E00F6180D20FCF74CFD2A
:10374000002E06D02C002020FCF746FD0134A642B6
:10375000F9D1944B188803F013FC2020FCF73CFDB2
:10376000404603F00DFC2020FCF736FD7F2F1AD8D1
:103770004046FFF78DFF6B2F53D06C2F57D06D2F26
:1037800000D182E06E2F00D187E06F2F56D0712FCD
:1037900000D18AE0722F00D18DE0FD224346733BB9
:1037A00013424BD059E02D20FCF716FD3E20FCF7CC
:1037B00013FD2020FCF710FD4046FFF769FF784B12
:1037C0001B685B787F241C40692F00D19EE06A2F24
:1037D00000D1A5E0642F00D1B7E0744C032D00D1D7
:1037E000C7E02368022B00D8C3E0FCF741FEFEF7D8
:1037F00073FF0028F2D0FEF777FA0500012800D108
:10380000ADE0022800D1ADE00428E7D1664B1B688B
:10381000002B00D1ADE0664A1360644B02221A60AF
:10382000DCE7644B1B681B68002B07D0C7E7614BC4
:103830001B68191F1A680B689A42C0D0684603F0CB
:103840004AF9574B1B68587800029B78184301309F
:1038500003F096FB2920FCF7BFFC682F35D1504BB5
:103860001B685C782820FCF7B7FC534B1B68102BB7
:1038700027D02000FDF770F82920FCF7ADFC484B5D
:103880001B685B787F241C40A1E74A4B1B681A1F0A
:1038900012681B689A42D1D291E7464B1B681A1FE7
:1038A00012681B689A42C9D989E7424B1B681B689A
:1038B000002BC3D083E73F4B1B681B68002BBDD197
:1038C0007DE7200003F05CFBD6E7672F00D076E7AA
:1038D000334B1A6893781B04517809060B4311790E
:1038E0000B43D47824021C432820FCF775FC324B90
:1038F0001B68102B06D02000FDF72EF82920FCF7BE
:103900006BFC67E7200003F03BFBF7E72820FCF7A0
:1039100063FC2000FFF7E2FE2920FCF75DFC5CE77A
:103920002820FCF759FC2000FFF7D8FE4020FCF7C8
:1039300053FC20010830214C00190004000C03F056
:1039400055FB2920FCF748FC47E72020FCF744FC06
:103950003C20FCF741FC2D20FCF73EFC3DE7FEF748
:10396000CFFC3BE70D4A80235B0011680B431360DB
:10397000D4E62020FCF730FC43465F3B022B03D803
:10398000684603F0A8F8C9E67B20FCF725FC202058
:10399000FCF722FCC2E6C046D06A0008981400205A
:1039A000901400208C14002084140020FC010020BE
:1039B000B4140020641400205014002010080020CB
:1039C00010B5FFF79DFE074B1B68002B08D1064B77
:1039D0001B681B789B00054A9B589847FEF70CFE16
:1039E00010BDC04698140020901400200000002054
:1039F00010B51B4A1368013313601A4B1A68111D66
:103A0000196019490B6853601A787F2313401B0112
:103A1000164AD3189B680B601B787E2B0BD8144A70
:103A20001268032A04D09B00124A9B58984710BD85
:103A3000FFF7C6FFFBE70E4B1B68032B06D00E4BB0
:103A40001B68002BF3D1FFF7D3FFF0E7FFF758FE19
:103A5000094B1B68002BEAD1FEF7CEFDEFE7C0460D
:103A6000841400206C140020901400201008002002
:0C3A7000FC010020000000209814002041
:103A7C00F0B587B001AA3C4B13CB13C211001A68E6
:103A8C000A601B790B71394C394BE418394B1B68A4
:103A9C00A34263D2384D374E2F003BE0FDF726FF93
:103AAC003FE0FFF79FFF28E0FEF710FE00280CD147
:103ABC0033681B787E2B1BD82F4A1268032A14D02C
:103ACC009B002E4A9B58984717E0FEF707F90128F0
:103ADC0008D00228ECD12A4A80235B0011680B43E2
:103AEC0013603BE0FEF706FCE2E7FFF763FF04E040
:103AFC003B68032B1FD0FFF775FF214B1B68002B76
:103B0C002CD11C4B1B68002B1AD00133194A1360A3
:103B1C00A34223D22B68002BC6D11A4B1B68042B53
:103B2C00BCD0144B1B681B787E2BBAD89B00134A55
:103B3C009B589847E1E7FFF7DDFDFEF757FDDAE705
:103B4C000D4B1B68032B0BD00B4B01221A6000236F
:103B5C000D4A13700D4A13600D4A136007B0F0BD87
:103B6C0001A802F0B2FFEFE7906D000810020020F0
:103B7C00000E002090140020FC010020000000200A
:103B8C0098140020481400202B150020B01400209D
:043B9C00841400206D
:103BA000F8B5274B1C68002C2ED1264B1B68190139
:103BB000254A5218D168C022120511420AD0234A60
:103BC0001168081D10601B011F4AD3189B684B60C9
:103BD0002000F8BD1B011C4AD3189A681C4B1A60C0
:103BE0001C4B01221A701C4D2F681C4C2668522356
:103BF0002B6023601A4B00221A60FFF73FFF2F60F3
:103C00002660184B1C68E3E70E4B186802010E4B48
:103C10009B18DA68C0231B0514001C401A4204D10B
:103C200080231843FEF720FBD2E76920FEF71CFB38
:103C3000044B1868FEF718FB0A4B1C68C8E7C0461F
:103C40009C14002070140020100800206414002030
:103C5000901400202B150020441400204014002054
:083C6000A014002098140020BC
:103C680070B50023384A1370384A1360384A136015
:103C78001500384E0EE0384B1B68FF2B24D86820FF
:103C8800FEF7EEFA344B1868FEF7EAFA304B1A687A
:103C98002E4B1A60314C2B682268934230D2FEF7C3
:103CA8002BF93378002BF6D0FEF7C6F900281FD081
:103CB8002B4B1B68002BDED12A4A1368191D116093
:103CC800254A12685A60E1E76720FEF7C9FA224CD4
:103CD80003202056FEF7C4FA0223E05EFEF7C0FA7E
:103CE80023681812FEF7BCFA2068FEF7B9FACDE788
:103CF800FEF74CFA002809D0FFF74EFF002800D045
:103D080070BD134B1A68114B1A60C3E7FEF702FA2D
:103D180000280AD0FEF7BCFA134B1B68002BEFD122
:103D28000B4B1A68094B1A60B4E70F4A0123116854
:103D38000B4313600D4B1A680D4B1A60044B1A683D
:103D4800024B1A60DCE7C0462B150020381400200F
:103D580040140020C01300203C140020441400200C
:103D68009C1400206414002098140020A41400203F
:043D7800A81400206B
:103D7C00F0B5DE4657464E464546E0B591B00BA928
:103D8C00B94B0A0013CB13C203CB03C206AAB74B21
:103D9C0013CB13C211001A680A609A888A809B7927
:103DAC008B7102AAB24B13CB13C21B881380B14B7D
:103DBC001A68B14B1A60FEF79DF8FEF7E5F900287A
:103DCC000DD1FEF7A5F9002805D1AC4A01231168E5
:103DDC000B43136018E10BA802F077FE14E1A54B1E
:103DEC001A68A54B1A6006A802F06FFEA44D2B684A
:103DFC001801A44C001903F0F3F80D20FCF7E6F9B8
:103E0C002B681A01A418E168C022120508001040A2
:103E1C000190114200D0FEE01B019A4AD3189C6815
:103E2C00994BE41A2405240D1B5D0125642B00D14C
:103E3C00D1E0954E24E00D20FCF7C8F9019D1FE060
:103E4C00914B1A195078000202341F5D0743282049
:103E5C00FCF7BCF9781C03F08DF82920FCF7B6F9B7
:103E6C0001352020FCF7B2F92020FCF7AFF9013422
:103E7C00854B1B5D642B00D1ADE00135072DDAD8E5
:103E8C00A0190004000C03F075F83A20FCF79EF919
:103E9C00305DFFF7F7FB335D1A006B3A0A2ACFD976
:103EAC00682B1AD0672B2ED0692B4CD06A2B57D08D
:103EBC00652BD6D12220FCF789F9734B1B195B7843
:103ECC009B46A31C98465B46002B7DD06E4B43440F
:103EDC0099465C460F239A466BE001342820FCF788
:103EEC0075F96A4B1B68102B08D0674B185DFCF7F3
:103EFC002DFD2920FCF76AF90135B2E7624B185DFC
:103F0C0003F06EF8F5E76048021993781B045178BA
:103F1C0009060B43D7783F020434025D13431F4359
:103F2C002820FCF753F9594B1B68102B07D038008D
:103F3C00FCF70CFD2920FCF749F9013591E7380015
:103F4C0003F04EF8F6E701342820FCF73FF94E4B0E
:103F5C00185DFFF7BDFB2920FCF738F9013580E728
:103F6C0001342820FCF732F9474B1F5D3800FFF76E
:103F7C00AFFB3F01083743483F184020FCF726F9B8
:103F8C003804000C03F02CF82920FCF71FF901353C
:103F9C0067E75C20FCF71AF9380902F088FD5046F7
:103FAC00384002F084FD013C01239C46E144002C86
:103FBC0009D04B461F783B00203B5E2BE9D83800DC
:103FCC00FCF704F9EFE7D8444446013C2220FCF707
:103FDC00FDF8033545E72C4820180004000C02F0CE
:103FEC00C9FF3A20FCF7F2F83B20FCF7EFF8244B22
:103FFC001A681201234B9B18DA68C0231B051A425E
:10400C0009D10D20FCF7E2F811B0F0BCBB46B2466A
:10401C00A946A046F0BD02A802F057FD1B4B1B6839
:10402C00102B18D0164B1A681201164B9B18986857
:10403C0002F0F9FD2020FCF7C9F84020FCF7C6F887
:10404C000F4B1868000108300E4BC0180004000C10
:10405C0002F0C6FFD5E70A4B1A681201094B9B18F0
:10406C00986802F0BDFFE5E7F06A0008046B0008F1
:10407C00186B0008401400203814002098140020FD
:10408C007014002010080020100200205014002092
:10409C00134B1B68134A1360134A1268120113491D
:1040AC005218BE20C000844661448A420AD210498C
:1040BC000139891A8908013189005118002001C27F
:1040CC008A42FCD10B4A934209D80B4A9B180B49E4
:1040DC008C4662440021197001339342FBD1704726
:1040EC00A8140020A4140020801400201008002024
:1040FC00000E0020FE05000010020020FF0500004D
:10410C0010B5164B1A68164B1A60FDF7F3FEFEF746
:10411C003BF800280DD0114B1A68114B1A60114B4B
:10412C001B68032B0BD8104A802311680B431360B8
:10413C0004E00D4A212311680B43136010BD0B4A98
:10414C0013600B4A1B0100219954D318DB681B0523
:10415C001B0D084A1360FFF79BFFEFE7401400208C
:10416C0038140020701400209814002080140020B3
:08417C0010080020A814002027
:1041840010B50023204A1360204A1360204A13709C
:10419400204A1360204A1360204A01211160204AFA
:1041A4001360204B1A68204B1A60204A00231178B0
:1041B400002903D0013310325F2BF8D11C4A13605D
:1041C4001C4A1D4BD35C642B1CD01B4B1100013BC0
:1041D400CA5C642A02D0002BF9D102E0002B00D083
:1041E4000133164A1360FFF757FF154A154B1A603F
:1041F40000231360144A0F491160144A1360FDF739
:10420400D1F910BD0C4BEBE7A01400209C14002046
:104214002B150020B014002084140020FC01002081
:104224004C1400207C14002050140020100800209E
:104234008014002010020020FF050000A8140020B4
:10424400F81200206C140020901400209814002010
:1042540030B5B9B036AAA04B1968369199889180C7
:104264009B79937134AA9D4B1968349199889180F4
:104274009B79937131AA9A4B03CB03C211001A881C
:104284000A809B788B702EAA964B13CB13C22BAA51
:10429400954B03CB03C211001A880A809B788B705C
:1042A40027AA924B13CB13C21B88138022A9904BCD
:1042B4000A0013CB13C203CB03C21CA98D4B0A0003
:1042C40013CB13C203CB03C21B78137018AA8A4BF7
:1042D40013CB13C21B68136014AA884B13CB13C2ED
:1042E4001B8813800FAA864B13CB13C211001A68C4
:1042F4000A609B888B8009A9824B0A0013CB13C2E6
:1043040003CB03C21B78137005AA7F4B13CB13C2D4
:104314001B78137001AA7D4B13CB13C21B88138027
:104324007B4B1A687B4B54339A4200D280E07A4923
:104334000423086803430B60764B0C339A4204D27F
:10434400754A042311680B431360744B1B68002BDC
:104354000FD0734B1968734B09010022CA545B18C0
:104364005A709A70DA701A715A719A71DA719A6085
:10437400DA606A4B00221A606B4B1B68002B0ED06C
:104384000024694D2020FBF725FF01342B68A3424C
:10439400F8D85E20FBF71EFF0D20FBF71BFF36A8A5
:1043A40002F097FB5C4C206802F0E8FD3D20FBF72F
:1043B40011FF2368DB075ED4574B1B689B075ED451
:1043C400554B1B685B075ED4534B1B681B075ED4BD
:1043D400514B1B685B065ED44F4B1B689B065ED437
:1043E4004D4B1B681B065ED44B4B1B68DB055ED430
:1043F400494B1B689B055ED4474B1B685B055ED429
:10440400454B1B681B055ED434A802F062FB464B87
:104414001868FCF79FFA2920FBF7DCFEFFF7B0FED3
:104424000D20FBF7D7FE414B00221A6039B030BD96
:10443400384B0C339A4200D282E7374B1B68002B6F
:1044440000D082E7354B1B68002B40D1384B1B68EA
:10445400012BE5D02020FBF7BDFE6F20FBF7BAFE51
:104464006B20FBF7B7FE334B1B68102BD8D14820C9
:10447400FBF7B0FED4E731A802F02BFB9CE72EA893
:1044840002F027FB9CE72BA802F023FB9CE727A85C
:1044940002F01FFB9CE722A802F01BFB9CE71CA870
:1044A40002F017FB9CE718A802F013FB9CE70FA887
:1044B40002F00FFB9CE714A802F00BFB9CE709A891
:1044C40002F007FB9CE705A802F003FB9CE701A8A8
:1044D40002F0FFFAA4E7C046586B0008606B0008BE
:1044E400686B0008746B0008806B00088C6B000814
:1044F4009C6B0008B06B0008C86B0008D86B000800
:10450400E86B0008FC6B0008146C0008246C0008BD
:10451400641400205C130020981400209C140020D4
:10452400801400201008002038140020B01400204B
:08453400A01400205014002027
:10453C0010B500231B4A13600A221B490A601B4951
:10454C000A601B4A012111601A4A13601A4A13604F
:10455C001A4A073111601A4A2A311160194A13603C
:10456C00013B194A1360194A1360194B3122562426
:10457C000021C02000051C705A709970D860996099
:10458C0010330132D2B2352AF5D1124B313A1A60BE
:10459C0000230F493C328B540F4A1360FFF7ECFD9C
:1045AC0010BDC046101500207C14002050140020B3
:1045BC00FC010020B81400205814002060140020C6
:1045CC005C14002094140020781400207414002033
:0C45DC001008002080140020A81400200B
:1045E80070B5164C164D2B682360FDF785FC2B68BB
:1045F8002360144B1D68013D28006B1C17D02D014A
:10460800114BED18114E10E08B420BD1002913D03D
:104618000132A95C935D1C00613C192CF4D8203B45
:10462800DBB2F1E7103D013804D30022F1E70120A5
:10463800404201E00120404270BDC04638140020CD
:10464800401400208014002010080020C01300200F
:1046580010B5FFF7C5FF0400431C0DD002011D4B28
:104668009B18DA68C0231B051A420BD01A4A80230C
:1046780011680B43136010BD174A212311680B43BF
:104688001360F8E7FFF7ACFF431C11D00201114B90
:104698009B18DA68C0231B051A420FD1844213D92C
:1046A8000C4B24011C19A268000118188260E2E76B
:1046B800094A212311680B431360DCE7064A80236B
:1046C80011680B431360D6E7034A802311680B4334
:0C46D8001360D0E71008002098140020A8
:1046E40010B5FFF77FFF431C0FD003010D4AD2180A
:1046F400D3681B051B0D0C495B1892689A420AD3B8
:104704000001084A1018836010BD084A212311686B
:104714000B431360F8E7054A802311680B431360C9
:10472400F2E7C04610080020100200209814002070
:10473400F8B506000D490A68571C0F6054783F19F4
:10474400002C10D00D0005E05878FBF743FD013C28
:10475400002C08D02B685A1C2A60012EF4D05878FB
:10476400FBF72CFDF3E7014B1F60F8BD901400200C
:10477400074B1A68511C196051780902901C186083
:1047840092781143802292050A431A607047C0460A
:04479400901400205D
:1047980010B5084B1B681B68002B08D0064A136825
:1047A80002331360034A1368043B136010BDFFF71C
:0C47B800DDFFF7E76414002090140020DF
:1047C40010B5094B1B68191F1A680B689A4208D167
:1047D400064A136802331360034A1368043B1360E8
:1047E40010BDFFF7C5FFF7E7641400209014002004
:1047F40010B5094B1B68191F1A680B689A4208DD2B
:10480400064A136802331360034A1368043B1360B7
:1048140010BDFFF7ADFFF7E76414002090140020EB
:1048240010B5094B1B68191F1A680B689A4208DAFD
:10483400064A136802331360034A1368043B136087
:1048440010BDFFF795FFF7E76414002090140020D3
:1048540010B584B001A8214B020012CB12C21B88F0
:10486400138002F036F91E4C2068FCF773F82368B5
:104874001F2B15D00B2B1DD0194B1B68132B20D0CD
:10488400174B1B68262B20D0154B1B68392B20D0C7
:104894003020FBF79FFC3020FBF79CFC04B010BDDC
:1048A4003220FBF797FC3520FBF794FC3020FBF714
:1048B40091FCF3E73520FBF78DFC3220FBF78AFCF3
:1048C400DAE73220FBF786FCDAE73420FBF782FCD8
:1048D400DAE73620FBF77EFCDAE7C046406C0008D6
:0448E400201500207B
:1048E80070B5A6B0B54B1A6824929A886946942088
:1048F80009180A809B796A4696215218137022ADCE
:10490800AF4B2A0003CB03C2AE4B1A6820929A8899
:104918006946842009180A809B796A4686215218BC
:1049280013701CACA84B220043CB43C21B781370F6
:10493800A64B1A681A929A881AAB9A80A44B1A68DE
:1049480018929A8818AB9A8014AAA24B43CB43C2F8
:104958001B68136011AAA04B43CB43C20CAA9F4B00
:1049680043CB43C211001A680A601B790B719C4B38
:104978001A680A921A790AAB1A7106AA994B43CB9C
:1049880043C21B88138003AA974B03CB03C21B782F
:10499800137001AA954B19680191998891809B79A8
:1049A8009371934B00934420FBF712FC6120FBF7B3
:1049B8000FFC7420FBF70CFC6120FBF709FC24A812
:1049C80002F085F88B480C3002F0D6FA280002F085
:1049D8007EF824A802F07BF8874802F0CDFA200080
:1049E80002F075F8854802F0C7FA20A802F06FF8BF
:1049F800834802F0C1FA0D20FBF7EAFB814B1B68E4
:104A0800002B10D11AA802F062F814A802F05FF87F
:104A180011A802F05CF87C4B1B680024002B06D020
:104A2800774E794D67E018A802F051F8EDE76E204F
:104A3800FBF7CEFB6F20FBF7CBFB6E20FBF7C8FB29
:104A48006520FBF7C5FB0D20FBF7C2FBFFF7FEFE59
:104A58006E4B1B6802229343012B02D00CA802F074
:104A680036F80D20FBF7B4FB0AA802F030F8684BC3
:104A78001868FBF76DFF2C20FBF7AAFB654B1B683A
:104A8800102B40D0644B1868FBF762FF2C20FBF713
:104A98009FFB624B1868FBF75BFF06A802F017F84C
:104AA8005F4B1E68002E3AD10020FBF751FF03A888
:104AB80002F00DF85B4B1868002800DA70E0554BDF
:104AC8001B68102B00D16FE0FBF742FF01A801F033
:104AD800FEFF554B1868002869DB4E4B1B68102BEE
:104AE80069D0FBF735FF0D20FBF772FB26B070BDD0
:104AF800FBF76EFB01342B68013B1B01F318185DB3
:104B08000028F5D19FE7444B186802F06BFA2C2077
:104B1800FBF75EFB414B186802F064FABDE77501CC
:104B2800AD1BAD00AD192D012900404802F084FAF3
:104B38000400FBF70DFF6643B404A41BA400A41BE8
:104B4800E400A4192401A41B6401394B9C46644465
:104B58002E20FBF73DFB2900200002F06DFAFBF741
:104B6800F7FE2900200002F0F2F98C0064186400B6
:104B78002900200002F060FA06002900200002F057
:104B8800E6F9880040184000290002F055FA04238D
:104B980083429B415B42F6183000FBF7D9FE86E75B
:104BA800684601F094FF91E702F01CFA8EE7684628
:104BB80001F08DFF97E702F015FA94E75C6E0008A4
:104BC800646E00086C6E0008746E0008846E00083D
:104BD8008C6E0008946E0008A46E0008B06E000881
:104BE800C46E0008CC6E0008DC6E0008E86E000891
:104BF8004F4646005C130020F812002010020020E7
:104C08001008002010150020B814002008150020F6
:104C18005814002050140020601400205C14002058
:104C2800941400207814002074140020006CDC0216
:044C380000389C1C88
:104C3C0030B58BB003A8124B020032CB32C232CB50
:104C4C0032C21B8813806A460E4B32CB32C201F043
:104C5C003CFFFCF781F80028FBD0FF2318405928B3
:104C6C0008D0684601F031FF0D20FBF7AFFA0020A9
:104C7C000BB030BD0D20FBF7A9FA0120F8E7C046B8
:084C8C0008630008246300081E
:104C9400F0B591B0040001A9334B0A0023CB23C221
:104CA40023CB23C223CB23C203CB03C22F4D304ECD
:104CB40033682B60FDF722F933682B60FDF7BEF9EA
:104CC400051E08D02B4A802311680B43136000256E
:104CD400280011B0F0BDFDF71FFA002804D10CA87C
:104CE40001002A00244F0EE001A801F0F2FEFFF7B4
:104CF400A3FF0028F3D10225EAE7002B12D0072AEC
:104D04000AD001320131D35D0B701E00613E192EB1
:104D1400F3D8203B0B70F2E7164A022311680B43C9
:104D24001360D5E70CAB1B78002B0CD0134A126828
:104D3400120113495218535501354378002B02D000
:104D44000130072DF7D10D4B1A6812010C4B9B183B
:104D54005D1900226A700B4A10680B4A82189A6027
:104D64002043D8600125B3E73063000838140020DD
:104D74004014002098140020C01300208014002048
:0C4D840010080020A814002010020020DD
:104D900070B5C0200005FFF77DFF00280DD00A4C3C
:104DA00022680A4803681D010949491915688D6080
:104DB000043A22600133036070BD064A0123116882
:104DC0000B431360F8E7C0466414002080140020F1
:084DD0001008002098140020D7
:104DD80010B50020FFF75AFF002808D0022807D096
:104DE800074B1A68074B1A60074B01221A6010BD5F
:104DF800064B1B681B01064A00219954F7E7C04679
:104E0800A8140020A41400209C1400208014002062
:044E1800100800205E
:104E1C0010B588B06946214B0A0013CB13C213CBD3
:104E2C0013C203CB03C21E4A13681C68043B1360F5
:104E3C00962C1BD0112C26D0192C03D113240B2CFF
:104E4C0018D002E0312C12D11F24132C12D01F2C9D
:104E5C0010D0262C0ED0392C0CD0602C0AD0114A34
:104E6C008023DB0011680B4313600AE06024382CAC
:104E7C000AD12624684601F028FEFFF7D9FE002847
:104E8C0006D108B010BD0B24572CD8D13924F1E72A
:104E9C00054B1C60FBF726F9F3E7C0465C63000882
:0C4EAC0064140020981400202015002041
:104EB80010B588B001A91B4B0A0013CB13C213CB42
:104EC80013C21B881380184A13681C68043B1360BC
:104ED800164B1B68A34208D0154B1B68002B06D045
:104EE800012C0DD813D0114B1C6008B010BD114A0D
:104EF800803311680B4313600C4B00221A60F4E7EF
:104F08000C4A8023DB0011680B431360EDE701A80E
:104F180001F0DDFD0D20FBF75BF9FFF78BFE0028A4
:104F2800E1D1E2E7806C0008641400200815002035
:084F38002C1400209814002045
:104F400030B585B0174B1A6802929A8869468A81F3
:104F50009B798B73144B1A6800929A888A809B798C
:104F60008B71FBF7C7FF114C23681D6802A801F085
:104F7000B2FDFCF72FFD2020FBF72EF923681C68FB
:104F8000684601F0A8FDFCF725FD2020FBF724F979
:104F9000FFF754FE002803D0054B1D60054B1C6035
:104FA00005B030BDF06E0008F86E000864140020F3
:084FB000BC14002014150020C0
:104FB80030B589B001A80B4B020032CB32C232CBDC
:104FC80032C21B68136001F082FDFFF733FE002830
:104FD80001D109B030BDFBF7A7FA034B01221A60D3
:0C4FE800F7E7C0467C63000810150020AD
:104FF40010B58CB006A91E4B0A0013CB13C203CB09
:1050040003C21B78137069461A4B0A0013CB13C2F0
:1050140003CB03C21B781370174A13681968043B47
:10502400136001290ED8002914D1684601F051FDFE
:10503400FFF702FE00280BD0104B00221A60FFF786
:105044007BFA05E00E4A8023DB0011680B431360F2
:105054000CB010BD06A801F03CFDFFF7EDFD0028E3
:10506400F6D0064B01221A600120FBF7C9F8EFE7DE
:10507400B06D0008C86D00086414002010150020ED
:04508400981400205C
:10508800074B1B68002B09D0054B00221A60054A04
:105098001368191D1160044A12685A607047C046A7
:0C50A800B014002064140020AC140020A0
:1050B40010B5214B1A68214B1A60FCF71FFFFDF74E
:1050C40067F8002821D01C4B1A681C4B1A601C4B33
:1050D4001A6812011B4B9B18DA68C0231B051A427D
:1050E40019D0194B1B78002B1BD1184B1B68002BB4
:1050F4001AD117480368124A11680901114A521853
:1051040019689160043B036004E0124AA02311680B
:105114000B43136010BD0F4A802311680B431360C7
:10512400F8E7FFF7AFFFE0E76A20FDF79BF8044BD1
:105134001868FDF797F8EDE74014002038140020B4
:1051440070140020100800202B1500209C1400204F
:085154006414002098140020EF
:10515C0010B50A4B1B78002B0DD1094A136809496D
:10516C0018680860043B1360FDF762FCFDF7E6FC71
:10517C00FDF73EFD10BDFFF781FFEEE72B1500207C
:08518C006414002094140020BB
:1051940010B50D4B1B78002B0DD10C4A13680C492C
:1051A40018680860043B13600A4B1B88DB0705D5AD
:1051B400FDF7C8FC10BDFFF765FFEEE7064B1822AC
:1051C4001A60FDF739FCF3E72B1500206414002066
:0C51D40078140020000400409414002017
:1051E00010B50D4B1B78002B0DD10C4A13680C49E0
:1051F00018680860043B13600A4B1B88DB0705D561
:10520000FDF7FCFC10BDFFF73FFFEEE7064B182251
:105210001A60FDF713FCF3E72B150020641400203F
:0C522000741400200004004094140020CE
:10522C00F0B5C64600B588B069462B4B0A0013CBC7
:10523C0013C213CB13C203CB03C2284B1B78002B16
:10524C0014D1274A13688024A40519680C43043B25
:10525C001360244B9C420CD9234A8023DB00116839
:10526C000B43136008B080BCB846F0BDFFF706FFD7
:10527C00E7E70D20FAF7AAFF684601F026FC2000AC
:10528C0001F078FE270080370F25032398460FE0A6
:10529C000D20FAF79BFF200001F06CFE3A20FAF784
:1052AC0095FF300001F039FC00250134BC420ED0D2
:1052BC0026780135102DEBD0300001F02EFC434642
:1052CC002B40032BF1D17C20FAF780FFEDE70D206A
:1052DC00FAF77CFFC6E7C046986300082B15002040
:0C52EC0064140020807F00209814002033
:1052F80082B03A4B1A6801210A431A605A68384842
:1053080002405A601A68374802401A601A683648DC
:1053180002401A605A68354802405A60DA6A0F201B
:105328008243DA621A6B324802401A635A6B8A4324
:105338005A6300229A6000920192196880225202F0
:105348000A431A60190080229202A020C0010B684B
:1053580013400193009B01330093019B002B02D162
:10536800009B8342F3D11D4B1B689B0306D5012389
:105378000193019B012B04D002B0704700230193D5
:10538800F7E71C4B11221A60144B5A685A605A6886
:105398005A605A6818490A405A6059688822520364
:1053A8000A435A601968802252040A431A60190095
:1053B800802292040B681342FCD0084B5A680321E0
:1053C8008A435A605A6801390A435A6019000C2204
:1053D8004B681340082BFBD1CEE7C04600100240B3
:1053E8000CB8FFF8FFFFF6FEFFFFFBFFFFFFC0FF53
:0C53F800ACFEFFFF00200240FF7FC0FF62
:105404004C4B80221A6000224B4B1A604B490868AF
:1054140080231B0203430B60494B1A601B68494AF3
:105424009A1849490A6049490A604949581849493A
:105434000860494958184949086049495818494970
:105444000860494958184949086049495818494960
:105454000860494958184949086049498C466344D9
:1054640048490B60484B1B68002B06D113001833C6
:1054740046490B60464902330B6040231380354B89
:105484001B6800221A80354B1B6880211980354B1C
:105494001B6840491980354B1B68802040001880E8
:1054A400344B1B681A80284B1B689881DA810130C1
:1054B400FF3018825A82314B1B681880314B1B68AD
:1054C4001980314B1B68002B0BD1304B1B68C0215A
:1054D400890019802E4B1B681A801B4B1B6899830B
:1054E400DA832D4B2D4A1A802D4B2E4A1A802E4BCF
:1054F4002E4A1A80244B1B68002B02D12C4B2D4AB8
:105504001A802D4BBF2212021A6000232B4A13600B
:105514002B4A13602B4A2C490A602C490A602C4AF6
:105524002C490A602C490A602C4A13702C4A1370C7
:105534007047C0464C5C004034140020585C004066
:10554400505C00400060004030140020F41400203F
:1055540002600040E014002004600040F8140020C1
:1055640006600040E414002008600040F0140020AD
:105574000A600040DC14002014600040EC14002099
:1055840016600040D814002028140020E8140020DD
:10559400D41400200084FFFF005C0040203200008F
:1055A400045C004031300000085C004032300000F0
:1055B4000C5C004033360000405C004014140020B2
:1055C4002C140020000E0020C8140020C414002055
:1055D400CC110020D0140020CC1400200111002094
:0455E4009112002000
:1055E80070B5204CE36980252D042B43E361FAF75D
:1055F8006FFD23691D432561FAF76AFD236B80223D
:10560800134323632369184A134023619022D20568
:10561800136816490B401360154B0021154A198071
:1056280002339342FBD1144B0021144A19800233F0
:105638009342FBD1124A116880231B020B4313606B
:10564800104C01232360C820FAF760FF0023236071
:10565800094A1360FFF7D2FE0B4B802212061A602C
:1056680070BDC04600100240FFFF7FFFFFFFC3FF71
:10567800005C0040205C0040445C0040605C0040EE
:0C568800585C0040405C004000E100E085
:1056940070B582B0284B1B68402B45D9274B1B683B
:1056A40040221A80244A1368403B1360234B1B6832
:1056B4001B88002B16D0224C002122481F4D036862
:1056C4001E785A1C02605A78023303601302334373
:1056D40023800234013189B22B681B8801335B10AB
:1056E4009942ECDB184B1B881B0604D5164A138819
:1056F40016490B401380164B1B68164A1A80124B2E
:105704001B889BB26A46D380D3889B0602D40E4B77
:10571400114A1A806B4606331B88DB0602D40A4BF7
:105724000E4A1A8002B070BD034B1968034A12680E
:10573400118000221A60B9E714140020E01400203C
:105744004060004020140020005C00400F8FFFFFE9
:10575400E41400200084FFFFA082FFFF9082FFFF7B
:1057640082B0174B1B6800221A80164B1B881B063D
:1057740004D5144A138814490B401380104B1B683A
:1057840000221A800F4B1B889BB26A46D380D388B1
:105794009B0602D40B4B0D4A1A806B4606331B88BA
:1057A400DB0602D4074B0A4A1A806B4606331B8871
:1057B4005B0402D5034B074A1A8002B07047C04607
:1057C400E0140020005C00400F8FFFFFA082FFFF69
:0857D4009082FFFF80C2FFFF7D
:1057DC0000B583B01C4A13881C490B4013801C4B2A
:1057EC001B68052B1DD01B4B1B68002B29D1164B9E
:1057FC001B881BB2002B1EDB134B1B889BB26A460B
:10580C00D380D3889B0402D40F4B134A1A806B4667
:10581C0006331B88DB0402D40B4B104A1A8003B0EE
:10582C0000BD0F4B1B68802213430E4A1360084BBC
:10583C0000221A60D7E7044A13880B490B401380E7
:10584C00DAE7FFF721FFEAE7005C00400F8FFFFF6C
:10585C00181400201414002080A2FFFF8092FFFF78
:0C586C00341400204C5C00408F0F000042
:1058780082B0134B1A8813490A401A801B881B06EA
:1058880004D50F4A138810490B4013800C4B1B8812
:105898009BB26A46D380D388DB0602D4084B0B4AF6
:1058A8001A806B46DA8806331B889B0402D4044BA3
:1058B800074A1A806B4606331B8802B07047C046F9
:1058C800005C00408F0F00000F8FFFFF9082FFFFEA
:0458D80080A2FFFFAC
:1058DC0030B587B0B74B1B881B0500D456E1B54AD1
:1058EC001388B5490B401380B44B1B78B4490B702B
:1058FC00B44B1A78B44B1A70B44B1A88B44B1A8048
:10590C001A88120AB34802701B88DBB2B24A1370B1
:10591C00B24B1A88B24B1A80B24B1A88B24B1A800F
:10592C00B24B00221A60B24B1B68B24A1A800B7839
:10593C00212B31D0A24B1B78DBB2A12B62D0A04B18
:10594C001A7861231A4206D09D4B1B7861221340B2
:10595C00012B00D017E1974A138897490B4013800D
:10596C00994B1A78D3B2062A00D17DE0062B66D863
:10597C00002B70D0052B00D0F6E09F4B00221A6054
:10598C00FFF7EAFE924B1B887F2213409B4A136061
:10599C00964B05221A6005E18B4B1B78202B0BD004
:1059AC00894B1B78222B2AD1824A138882490B40BF
:1059BC001380FFF7D1FEF5E07E4B1B889BB21622BD
:1059CC006A44138013889B0402D47A4B8C4A1A8045
:1059DC0016236B441B88DB0402D4764B894A1A804D
:1059EC0016236B441B885B0403D5724BA0229200D8
:1059FC001A80704A13881BB2002BFBDBD2E0FFF736
:105A0C0035FFCFE0704B1B78212B98D1694A138856
:105A1C0069490B401380784A07231360724B1B882B
:105A2C009BB21268934204D26F4B1B889BB2724A92
:105A3C001360754B754A1A60FFF726FEB2E0092B0E
:105A4C0000D091E06C4B00221A60FFF785FE704B82
:105A5C00FF221A60A6E0684B02221A606A4B6D4A5C
:105A6C001A60FFF711FE9DE05A4B1B78012B1DD0DD
:105A7C00584B1B78022B53D0564B1B78032B70D1F1
:105A8C00554B1B78012B69D15B4A17331360564B6E
:105A9C001B889BB21268934204D2534B1B889BB257
:105AAC00554A1360584B5C4A1A6028E0524B12223C
:105ABC001A605A4B1B68012B24D0594D524B1D6058
:105ACC00584B1C68584A012394421DD0681E6A46E4
:105ADC00D11CC25CCA540133132BFAD101AB1C721A
:105AEC00240A5C72514B9D4215D0514B1A7801AB74
:105AFC009A724F4A1268120ADA72434A1360FFF71D
:105B0C00C3FD4FE0494DD9E74A4B494A12689A42C6
:105B1C00F5D00123DAE7464B1A680332D2B2E6E736
:105B2C003E4B1B68012B12D0334B43221A60364B71
:105B3C00414A1A602C4B1B889BB22F4A1268934225
:105B4C00DDD2294B1B889BB22B4A1360D7E72A4B1B
:105B5C0065221A602C4B394A1A60EBE7FFF786FE78
:105B6C0020E0FFF783FE1DE0154B1B78002B02D0C5
:105B7C00FFF77CFE16E00F4A13880F490B40138089
:105B8C00FFF7EAFD0EE0FFF771FE0BE0094B1B88F7
:105B9C009BB216226A44138013881BB2002B03DBC2
:105BAC00FFF7DAFD07B030BD1388034A1340014AF2
:105BBC001380F5E7005C00408F0F00008060004010
:105BCC0026150020816000402715002082600040CF
:105BDC0002110020281500202915002084600040A7
:105BEC00241500208660004092120020181400201A
:105BFC00E41400200084FFFF14140020341400204F
:105C0C0080A2FFFF8092FFFF20140020446F000849
:105C1C002C140020C06C0008AC690008281400206B
:105C2C00A46C0008BC14002083040000D06C000895
:105C3C001415002040570000006F0008EC6D0008A0
:105C4C00F0B5DE4657464E464546E0B583B03C4B74
:105C5C001B881B0604D53A4A13883A490B4013801B
:105C6C00394C0022394FB846394B9C46BA46B94696
:105C7C0033E05346374E1E6044E001AB1B882B804B
:105C8C005A46354B1B681A802D4B1B889BB26A46B3
:105C9C00D380D3889B0602D4294B304A1A806B469A
:105CAC0006331B88DB0602D4254B2D4A1A8003B021
:105CBC00F0BCBB46B246A946A046F0BD254B2349D5
:105CCC000B600232D2B26B46598801AB1B880902B9
:105CDC000B432B80402AD4D00234A51E3B682149AB
:105CEC0008688342CDD0694600264E8019788B46D1
:105CFC0001A95E460E80013341460B60614609687E
:105D0C008B42B6D0531CDBB29B46402BB5D04B46D6
:105D1C001B6883420AD01878834668465E464680E4
:105D2C0001339942CAD009490B60CAE76B465A88BD
:105D3C0001AB1B88120213432B805A46CCE7C0469A
:105D4C00045C00400F8FFFFF02610040C414002070
:105D5C0000020020000E0020DC140020A180FFFFB8
:085D6C009180FFFFC814002024
:105D740082B0114B1B881B0604D50F4A13880F49A8
:105D84000B4013800E4B1B6800221A800A4B1B88A1
:105D94009BB26A46D380D3889B0602D4064B094A39
:105DA4001A806B4606331B88DB0602D4024B064A74
:105DB4001A8002B07047C0460C5C00400F8FFFFF92
:0C5DC400D4140020A386FFFF9386FFFF8D
:105DD00010B5204B1B68002B34D01F4B18680028CF
:105DE0002FD01E4B1A681E4B1B689A4230D0511C94
:105DF0001A48016014781B4A1268914225D0174A4C
:105E00001268991A934201D2C433991A164B1B682F
:105E1000002B11D07D290FD8134B00221A60134B91
:105E20001B889AB29B0402D4104B11491980D304E9
:105E300002D40E4B0F4A1A80FAF742F98020000272
:105E4000204310BDFAF714FBC7E70B490160D6E702
:105E50000020F6E70C1500202C140020CC140020A4
:105E6000D0140020040200201C140020085C004014
:0C5E700082A0FFFF8290FFFFCC110020F9
:105E7C0070B5634B19684A1C1A60012800D1B9E04F
:105E8C000A788B1C5E4C2360022800D1B4E04D785C
:105E9C00CB1C2360032800D1B0E08E780B1D23604F
:105EAC000438C0B2931E0D2B00D9A4E0052A32D0C1
:105EBC000F2A30D013000C3B012B3DD904231400C6
:105ECC009C43022C5AD0C978072A7AD84D4B002211
:105EDC001A704D4B1A68541C1C6015701A684B4B89
:105EEC001B689A4269D0484B1A68541C1C60167087
:105EFC001A68464B1B689A4278D0434B1A68541C5C
:105F0C001C6011701A68414B1B689A4273D13E4B4E
:105F1C003F4A1A606FE03B4B00221A703A4B1A68EA
:105F2C00511C196015701A68384B1B689A4262D163
:105F3C00354B374A1A605EE0324B1B78AB420BD0C4
:105F4C00314B1A68511C196015701A682F4B1B685D
:105F5C009A420FD02B4B1D702B4B1A68511C196099
:105F6C0016701A68294B1B689A4244D1264B284A52
:105F7C001A6040E0244B264A1A60EBE7214B0022C2
:105F8C001A70214B1A68511C196015701A681F4B36
:105F9C001B689A420DD01C4B1A68511C1960167064
:105FAC001A681A4B1B689A4225D1174B184A1A606B
:105FBC0021E0154B164A1A60EDE7134B144A1A6090
:105FCC0091E7104B1B78AB428DD00F4B1A68541CC9
:105FDC001C6015701A680D4B1B689A4202D0094B55
:105FEC001D7080E7084B0A4A1A60F8E7064B084A0E
:105FFC001A6082E7002070BD0020FCE70020FAE761
:10600C002414002091120020D0140020040200203F
:04601C00CC11002083
:1060200070B582B0404B1B881BB2002B11DB3F4B7D
:106030003F4A1A603F4B1B6818783F4B1B685A0059
:10604000D21890423FD940283DD83C4D374C2600CD
:1060500025E0354A13883A490B401380E7E7FFF7FC
:106060000DFF14E0374B02221A600BE0364B1A6822
:10607000511C19603168097811701A68334B1B681C
:106080009A421CD02368013323600138C0B22A4BE6
:106090001B685A00D218904215D9402813D8012BFA
:1060A000DDD02B68022BE1D0204B1B681B78022B24
:1060B000D8D0042BDAD1234B04221A60E2E7224B1A
:1060C000234A1A60DEE7234B1A681F4B1B689A426B
:1060D00020D99B1AC4339BB201AA13801E4B002205
:1060E0001A6001AB1B889BB27E2B18D80E4B1B8805
:1060F0009BB26A46D380D3889B0402D40A4B174ACA
:106100001A806B4606331B88DB040BD4064B144AFB
:106110001A8007E09B1A9BB201AA1380DEE70E4BA0
:10612000FF321A6002B070BD085C004024140020E9
:1061300000620040D8140020281400200815002018
:106140008F0F000048140020D0140020040200200B
:10615000CC110020CC1400201C14002082A0FFFFD2
:046160008290FFFF2B
:1061640000B585B0234B1A6801921B681B0429D51E
:10617400019A0F2313400393019A102313400293AF
:10618400039B012B0BD0039B022B0BD0039B002BF7
:106194000ED1029B002B08D1FFF71EFB1DE0FFF779
:1061A40053FD1AE0FFF73AFF17E0FFF795FB14E001
:1061B400039B032B11D1104B1B68002B0DD1FFF750
:1061C400D7FD0AE00B4B1B685B0508D4094B1B6821
:1061D4001B050AD5074B094A1A6005B000BDFFF735
:1061E4000FF9044B064A1A60F7E7024B054A1A6096
:1061F400F3E7C046445C004028140020FFF7FFFF8B
:08620400FFFBFFFF7F8000009B
:10620C0070B5134B1B68002B21D0124B1A68511C14
:10621C00196010701A68104B1B689A4204D00F4E0C
:10622C000C4DAC24A4000AE00A4B0D4A1A60F6E7A8
:10623C00C02189008C466344991AA14207D9FAF708
:10624C0011F932682B68991A9A42F6D9F0E770BDA9
:10625C002C140020C814002000020020C4140020BC
:04626C00000E002000
:10627000074B1B68002B00DBFEE7054A11688023F3
:106280001B060B4313608369023383617047C0466A
:046290002CED00E011
:10629400555342206173207669727475616C204392
:0462A4004F4D3D001D
:1062A80043466F72746820666F722053544D3332C0
:1062B8004630343220762E0020286329323032309E
:1062C8002D323420572E536368656D6D65727400E6
:0862D800202D3E444247200046
:0862E0004B65726E656C3A001B
:1062E800A4300008FA300008883100088831000816
:1062F8000C3100081E310008303100085C310008FC
:1063080020636F6E6669726D20772E757070657286
:106318002063617365202759270000002063616EA0
:0863280063656C6C65642000E4
:10633000205761726E3A2077696C6C206F766572B7
:1063400072696465204B65726E656C204F502077D2
:0C6350002E73616D65206E616D6520008C
:10635C00426175642052617465206368616E676583
:10636C007320696D6D6564696174656C79212000B9
:10637C00536176652061637475616C20776F726B05
:0C638C0020696E20466C617368203F00A1
:10639800313238205352414D20627974657320732D
:1063A80074617274696E672066726F6D2030780050
:1063B80000000000000000000000000000000000D5
:1063C80000000000000000000000000000000000C5
:1063D80000000000000000000000000000000000B5
:1063E80000000000000000000000000000000000A5
:1063F8000000000000000000000000000000000095
:106408000000000000000000000000000000000084
:106418000000000000000000000000000000000074
:106428000000000000000000000000000000000064
:106438000000000000000000000000000000010053
:10644800000005000000000000000000000000003F
:106458000000000000000000000000000000010033
:10646800000004000000040000000000000000001C
:106478000000000000000000000001000000000013
:106488000000000000000000000000000000000004
:1064980000000400000004000000040000000000E8
:1064A80000000000000000000000000000000000E4
:1064B80000000000000000000000000000000000D4
:1064C80000000400000000000000050000000500B6
:1064D80000000500000004000000040000000400A3
:1064E800000004000000000000000100000001009E
:1064F800000001000000010000000300000003008C
:106508000000030000000300000003000000030077
:106518000000030000000300000003000000030067
:106528000000030000000300000002000000020059
:10653800000002000000020000000200000001004C
:10654800000001000000080000000800000008002A
:106558000000080000000800000008000000080013
:106568000000080000000800000008000000080003
:1065780000000800000008000000080000000800F3
:1065880000000800000008000000020000000200EF
:1065980000000100000001000000010000000100EF
:0C65A800000005000000010000000100E0
:1065B4004552524F5200000044524F500000000018
:1065C40044555000000000005357415000000000A3
:1065D4004F56455200000000524F54000000000086
:1065E4002D524F54000000005049434B000000005E
:1065F400524F4C4C00000000494E4A4543540000A1
:106604002B00000000000000312B000000000000FF
:106614002D00000000000000312D000000000000EB
:106624004142530000000000534849465400000012
:10663400414E4400000000004F52000000000000E2
:10664400584F5200000000004E4F5400000000005C
:106654002B2F2D00000000002A0000000000000085
:106664002F000000000000002A2F0000000000009E
:106674004D4F4400000000002F4D4F440000000027
:1066840052414E444F4D00003D3D000000000000CB
:10669400213D0000000000003E000000000000005A
:1066A4003E3D0000000000003C000000000000002F
:1066B400553C0000000000003E3D000000000000CA
:1066C400303D000000000000564152434F4E000090
:1066D40052455600000000004B45593F00000000A1
:1066E4004B45590000000000454D4954000000008E
:1066F4002E000000000000002E48000000000000F2
:106704002E440000000000002E22000000000000C3
:10671400445A000000000000485800000000000037
:1067240052583F00000000005258000000000000D2
:1067340054580000000000004E54580000000000AF
:106744005458220000000000584E4F500000000032
:106754004D530000000000004453000000000000FE
:10676400544958000000000054494D450000000001
:10677400465245510000000050574D3100000000C2
:1067840050574D32000000004F4800000000000048
:106794004F4C00000000000049505500000000006C
:1067A4004950440000000000495A00000000000065
:1067B4005244494E0000000052414443000000008E
:1067C400494E492D535049005350490000000000E0
:1067D4002E5300000000000046530000000000009B
:1067E4004F50530000000000555345520000000074
:1067F40053454500000000004D454D0000000000D9
:10680400535400000000000052554E0000000000E8
:106814004E4F2D4442470000444542554700000076
:10682400464F52474554000041424F525400000025
:106834005245504C41434500524553544F52450034
:106844004946000000000000434153450000000099
:106854003C434153450000003E4341534500000082
:10686400454C5345000000005448454E00000000CC
:10687400444F000000000000554E54494C000000F5
:106884005748494C45000000414741494E0000002B
:10689400464F5200000000004C4F4F5000000000D3
:1068A4004900000000000000434F4E54490000001E
:1068B400425245414B0000005A425245414B0000B0
:1068C40052455455524E00003A00000000000000AA
:1068D4003B00000000000000646F535452000000AD
:1068E400646F494F53545200646F4C495400000084
:1068F400646F4C4954384200646F56414C5545000E
:10690400646F524556000000646F49460000000061
:10691400646F434153450000646F3C434153450059
:10692400646F3E4341534500646F454C534500003A
:10693400646F444F00000000646F554E54494C008E
:10694400646F5748494C4500646F414741494E00C4
:10695400646F464F520000004C4F4F50000000003F
:1069640052502D310000000052502D340000000020
:106974004155544F455845004241554400000000DC
:1069840053504C49540000005649445049440000B7
:106994003F00000000000000534156450000000085
:0869A4004C4F414400000000CB
:1069AC001803430046006F007200740068002D004D
:0869BC004D00490044004900B0
:1069C400FEE7FEE7FEE7FEE7FEE7FEE7FEE7FEE79B
:1069D400FEE7FEE7FEE7FEE7FEE7FEE7FEE7FEE78B
:1069E400FEE7FEE7FEE7FEE7FEE7FEE7FEE7FEE77B
:1069F400FEE7FEE7FEE7FEE7FEE7FEE7FEE7FEE76B
:106A0400FEE7FEE7FEE7FEE7FEE7FEE7FEE7FEE75A
:106A1400FEE703488546FEF76DFC03E0704700007F
:046A24000018002036
:106A280011488546114C20680434004201D0804743
:106A3800F9E70F480F49091A082903DB0022026009
:106A4800043001600C480D49884205D002680430C2
:106A580003B4904703BCF7E700208646EC460020C5
:106A68000021074A9047FEE700180020A870000898
:106A78003015002078160020F96C0008F96C000821
:046A88004D0B0008AA
:106A8C0004207146084202D1EFF3088001E0EFF3D5
:0C6A9C00098001490847000071620008F1
:106AA800756E646572666C6F77212000202D2D2D20
:026AB8002000BC
:106ABA0010B502003030C0B2392801D93732D0B20D
:066ACA00F9F785FB10BD89
:066AD0002849502D3E0094
:106AD60010B5441C0078002806D0F9F77AFB01347B
:0A6AE600631E18780028F8D110BDD7
:106AF00063616E277420534545204B65726E656C4B
:106B00004F707300557365724865616465725F53B9
:106B100074727563743D0000566172436F6E3A562D
:066B2000616C75653D008B
:106B260010B5040003061B0F18003030392801D9B0
:106B360037331800F9F74DFB0F20044020003030A2
:106B4600392800D90730F9F744FB2020F9F741FB33
:026B560010BD70
:106B58004572726F722300002028636F6C2000005A
:106B6800206E6F7420666F756E6400005F53796ED7
:106B780074617820457272005F537461636B2045BD
:106B8800727200005F436F6D70696C65206F6E6C88
:106B9800790000005F4E6F20492F4F20436F6D6DC5
:106BA80020416363657373005F496E76616C696445
:106BB80020436F64652061636365737300000000A0
:106BC8005F6F7574206F6620436F6E74657874000C
:106BD8005F52756E74696D65206F6E6C7900000088
:106BE8005F5468726561642063616E63656C6C658F
:106BF800640000005F4E756D626572206F757420C9
:106C08006F662052616E6765000000005F44697618
:106C18002E6279205A65726F000000002020636F91
:0A6C28006D70696C696E672E2E0016
:0E6C320010B5F9F790FE2020F9F7CDFA10BD4D
:0A6C400042617564526174653D0005
:106C4A002F280FD90300303BDBB2092B08D90A29B8
:106C5A000BD00300413B052B0AD83738C0B2704726
:106C6A001800FCE701204042F9E701204042F6E71C
:066C7A0001204042F3E797
:106C80005553415254205465726D696E616C206792
:0A6C9000657473206C6F73742100AB
:0A6C9A0010B50120FBF7BDFD10BD91
:106CA4001201000200000040830440572404000045
:026CB4000001DD
:0A6CB60010B50020FBF7AFFD10BD84
:026CC0000000D2
:0E6CC20010B56B20FBF7CFFAFCF7A5FC10BD58
:106CD0001201000200000040830443572404000115
:026CE0000001B1
:0E6CE20010B56C20FBF7BFFAFCF795FC10BD57
:096CF00028566172436F6E3D00ED
:0E6CFA0010B56D20FBF7B3FAFCF789FC10BD56
:106D0800203C2D6E6F742061204B65726E656C207F
:106D18004F50206E6F722061206E756D6265720033
:106D2800203C2D696E76616C696420666F72204222
:106D380061636B2D4374726C00000000203C2D527F
:0D6D4800756E74696D65204572726F720082
:0E6D560010B56E20FBF785FAFCF75BFC10BD54
:106D640020202841444320696E69742920000000D2
:0D6D7400202028414443206F66662920003E
:0E6D820010B57120FBF76FFAFCF759FC10BD3D
:106D90002064656275672066696E69736865642042
:016DA00000F2
:0E6DA20010B57220FBF75FFAFCF749FC10BD3C
:106DB0004C6F616420466C6173682050726F6A6525
:106DC0006374203F000000004C6F616420456D70CB
:0D6DD00074792050726F6A656374203F0073
:0E6DDE0010B57320FBF741FAFCF72BFC10BD3B
:106DEC000902650002010080310904000000010164
:106DFC00000009240100010900010109040100023D
:106E0C0001030000072401000141000624020101D6
:106E1C0000062402020200092403010301020100FE
:106E2C00092403020401010100090581024000004C
:106E3C0000000525010103090502024000000000C5
:056E4C00052501010114
:0A6E520010B50120FDF76DFC10BD26
:106E5C00537461636B3D00002052657475726E0053
:106E6C0020557365723D000020436F646554687251
:106E7C006561643D00000000456D70747900000090
:106E8C00466C6173680000005F50726F6A656374D2
:106E9C00206C6F61646564002020204155544F457F
:106EAC0058453D002852533233323D5465726D695A
:106EBC006E616C29000000005350493D0000000039
:106ECC00202054696D65723A467265713D00000070
:106EDC00487A2050574D313D000000002C50574D42
:036EEC00323D0034
:0F6EF000564944203D200000504944203D2000D9
:106F0000090243000201008031090400000102026D
:106F100000000524001001052401030004240207D9
:106F20000524060001070583031000400904010041
:106F3000020A000000070581024000000705020266
:036F40004000000E
:076F440000C201000000087B
:0A6F4C0010B50020FDF7F0FB10BDAA
:106F56000A0010D00300400800E052008242FCD92B
:106F6600002000E05208934200D39B1A40418A4217
:0A6F7600F8D11900704700207047A1
:106F800010B50400000F16D12001000F17D1200208
:106F9000000F18D12003000F19D12004000F1AD1BF
:106FA0002005000F1BD12006000F1CD10F20204010
:106FB000FFF783FD10BDFFF780FD2001000FFFF7F5
:106FC0007CFD2002000FFFF778FD2003000FFFF784
:106FD00074FD2004000FFFF770FD2005000FFFF780
:0C6FE0006CFD2006000FFFF768FDDFE7E6
:106FEC0010B504003020F9F7F1F87820F9F7EEF835
:086FFC002000FFF7BFFF10BDEC
:10700400CA1751408B1A17D0C1174A4004B44840DC
:10701400411A48081A0000E052008242FCD90020BC
:1070240000E05208914200D3891A40419A42F8D1B3
:0C70340004BC5040801A704700207047D8
:107040000A000FD00300400800E052008242FCD941
:10705000002000E05208934200D39B1A40418A422C
:08706000F8D1704700207047D1
:10706800CA1751408B1A19D0C11706B44840411AA3
:1070780048081A0000E052008242FCD9002000E0D3
:107088005208914200D3891A40419A42F8D10CBC67
:1070980053405840C01A5140891A70470020704721
:1070A800D9720008100200201C130000EF720008BB
:1070B80000000020C8700008100200000000000056
:1070C8008D0E00089D0E0008C50E0008F50E00087C
:1070D8000D0F0008210F0008450F0008690F000870
:1070E800A90F000809100008691000088510000899
:1070F80095100008B1100008C1100008D910000848
:10710800211100083D1100085911000875110008E7
:107118008511000895110008B1110008E91100084F
:10712800211200085912000899120008B11200082B
:10713800D112000805130008291300084D13000890
:107148007113000891130008F1120008914D00080E
:10715800B55000083527000831190008E118000863
:107168008D190008D5190008BD1B00089B6C000884
:10717800B5130008D5130008F5130008B129000855
:10718800D51B0008FD1B0008B76C0008491400084F
:10719800F5290008252A0008711400088D14000834
:1071A8005D51000895510008E1510008A52D00081F
:1071B8000D2E0008792E0008D52E0008312F000862
:1071C800052D0008213000084932000885320008E2
:1071D800F5190008A9150008511C0008B91A00087B
:1071E8007D3D00082D520008C9150008D515000876
:1071F800E1150008F91800080D410008854100084C
:1072080059460008E5460008C36C0008E36C00080E
:10721800FB6C0008576D00084D240008AD140008E9
:1072280095240008836D0008A36D0008DF6D000831
:10723800C1240008ED240008E114000829170008FB
:10724800FD1400081115000839150008D94D00086B
:1072580045250008536E00084D6F0008ED1500081D
:107268002D1600084D1600087916000899470008E1
:10727800C5470008F547000825480008A516000876
:10728800C91600085917000891170008F9160008D0
:10729800C917000819180008C1180008D1180008F3
:1072A800112200081D4E0008B94E0008414F000881
:1072B800E9480008B94F0008F54F00080100000030
:1072C8000011002090120020C8110020006CDC0280
:1072D800206861680834094204D000220270013035
:0672E8000139FBD17047E3
:1072EE0020686168A2680C34124205D00B780370D6
:0A72FE0001300131013AF9D1704767
:0400000508006A176E
:00000001FF
